:0200000270008C
:10100000000001205D130700451307004713070088
:10101000491307004B1307004D13070000000000A1
:10102000000000000000000000000000113F070069
:101030005113070000000000531307005513070069
:1010400057130700571307005713070057130700DC
:1010500057130700571307005713070057130700CC
:1010600057130700571307005713070057130700BC
:1010700057130700571307005713070057130700AC
:10108000296107005713070057130700571307007C
:101090005713070057130700459007005713070021
:1010A000571307005713070057130700571307007C
:1010B000571307005713070000000000000000004E
:1010C000571307005713070057130700571307005C
:1010D000795A070057130700571307000000000054
:1010E0000000000000000000000000000000000000
:1010F00000000000000000000000000000000000F0
:1011000000000000000000000000000000000000DF
:1011100000000000000000000000000000000000CF
:1011200000000000000000000000000000000000BF
:1011300000000000000000000000000000000000AF
:10114000000000000000000000000000000000009F
:10115000000000000000000000000000000000008F
:10116000000000000000000000000000000000007F
:10117000000000000000000000000000000000006F
:10118000000000000000000000000000000000005F
:10119000000000000000000000000000000000004F
:1011A000000000000000000000000000000000003F
:1011B000000000000000000000000000000000002F
:1011C000000000000000000000000000000000001F
:1011D000000000000000000000000000000000000F
:1011E00000000000000000000000000000000000FF
:1011F00000000000000000000000000000000000EF
:10120000314932480A1A02D0072291438D463049AB
:1012100030480A1A06D00722914381F30988022236
:1012200082F314882C482D492D4A00F03CF82D48B3
:101230002D492E4A00F037F82D482E492E4A00F04D
:1012400032F82E482E492F4A00F02DF82E482F490B
:101250002F4A00F028F82F482F49304A00F023F891
:101260002F483049304A00F01EF8304830490022FB
:1012700000F024F82F483049002200F01FF82F4AD0
:1012800090471F481F49884205D00268043003B4C4
:10129000904703BCF7E700208646EC46002000217B
:1012A000274A9047FEE7884207D0521A05D00378B4
:1012B00001300B700131013AF9D17047884202D0F8
:1012C00002700130FAE770470000012000F80020AA
:1012D0000000012000000120E8D007007C59002018
:1012E000D0590020B8130700B8130700AC950700C9
:1012F000E8D007007C5900207C590020AC960700FC
:10130000AC960700AC960700AC960700AC960700B9
:10131000AC960700AC960700AC960700E6D0070035
:101320003CD10700D0590020D0590020D0590020CE
:10133000D8A10020D8A10020D8A100208513070043
:101340006D420700FEE7FEE7FEE7FEE7FEE7FEE789
:10135000FEE7FEE7FEE7FEE700F002B8FFF7FCBF9E
:101360000F484FF00701884385460E4880470E48D6
:10137000016841F470010160BFF34F8FBFF36F8FBD
:10138000FFF73EBF09480A490A4A884207D0521A65
:1013900005D0037801300B700131013AF9D1704763
:1013A000000001203562070088ED00E098960700F4
:0813B000685900207C5900205F
:1013B8007047000007B5044B0093044A402300F02F
:1013C80032F803B05DF804FBD9130700D1590020A7
:1013D8002DE9F84388461446B2B10F4B0F4E03254A
:1013E800002743F00109224608EB0701002003F01B
:1013F800C9FF0744241A48B933782BB14FF47A400F
:10140800C847013D02D13570BDE8F8830123337028
:10141800002CE8D1F8E700BFB0960700D0590020AB
:10142800704703F0DFBFF0B595B01D461646084675
:101438000C4601F02AFD1A9B0D93CDE9086500259D
:101448002B46082205A920460A958DF82C500C95A4
:1014580001F042FD079B0293069B03939DF814300D
:101468008DF8115003F00302012A1DD1BDF8142094
:10147800059DC3F3C203C2F383168DF81030B20082
:1014880008230EA9204601F027FDC5F3952508ABD2
:101498000093324602AB0EA9284600F0DFFB204637
:1014A80001F0F7FC15B0F0BD022AF8D1BDF81650CE
:1014B800C3F3C203C5F389158DF810300827082D2A
:1014C8002E4628BF08263B4632460EA9204601F084
:1014D80003FDAD1B08AB02AA31460EA8374400F045
:1014E80021FC002DEBD1DAE708B5FFF79AFF074892
:1014F800042100F01FFB002803DA0549412000F011
:10150800A1FD044B01225A7108BD00BF589607007F
:10151800C49607007C590020037813F0040216D003
:1015280003F00303012B03D0022B09D001207047DD
:101538000A6800880232C0F3831002440A60F5E7A3
:101548000B684288023303EB92130B60EEE71046F8
:10155800704700002DE9F04FDFF834A187B00F463F
:1015680000230446861C0DF1070015468DF8073048
:1015780000F0FCFCDAF804203A60DAF80830424F50
:1015880003F580639B1AA7F10409A7F10808B34281
:101598001BD30020002D72D004F00F039B0143F0F1
:1015A800050363F30F00DAF80430C3F309020332CA
:1015B80033444AF822009DF80700CAF8043000F0C6
:1015C80005FD012007B0BDE8F08F0121384600F085
:1015D8002AFE484600F042FE404600F03FFEDAF898
:1015E80008000290C0F3090003300AEB800002A94A
:1015F800FFF792FF029B8346C8B9C3F309020AEBBF
:101608008202D16803919A1C0133C3F309030AEBE0
:1016180083030292D86801F00303012B27D0022B21
:1016280008D01A494FF4C27000F00CFD0CE0C3F367
:101638000900D9E7BDF80E30C3F3891303334FEA25
:10164800104B02EB93030293404600F00AFE10B1E0
:10165800029BCAF808305946384600F0E4FDDAF82B
:101668000830DAF8042003F580639B1A8FE7BDF889
:101678000C30C3F383134FEA104B1344E3E7A4057C
:1016880044F006008FE700BF006B00206297070058
:10169800E45A0020064B074810B500221A7001F0E2
:1016A800ADFB044610B9044801F02AFC204610BDE1
:1016B800E45A0020309607000098070030B50A4C1D
:1016C80071B10A4A0A49121BD20800239A4201D171
:1016D800002030BD31F82350854202D00133F5E7B0
:1016E800034654F83300F4E7C09507003096070026
:1016F80068590020094B013903EBC000032909D8B8
:10170800DFE801F00A0204060420704700797047F8
:10171800407970470020704702207047C095070045
:10172800034BD3E90130C31A58425841704700BFF0
:10173800E45A00202DE9F04387B0FFF7F1FF064691
:10174800002840F0F080794C04F58055A861BFF37B
:101758004F8FA3680293C3F30903033304EB830099
:1017680002A9FFF7D9FE029B10B1AA69002A5DD031
:10177800C3F30902991C013304EB8202C3F3090382
:1017880004EB8303D268DB68049302F00303022BA3
:101798000392029155D1BDF80E306548C3F38918FC
:1017A8004746502F28BF502707F1080167F38F13CA
:1017B800C1F30901ADF80E3001F038FB06460028E8
:1017C80000F09D8001F061FB0023082203A9304648
:1017D80001F06EFB0299CB43C3F309030133C1F354
:1017E80009010331B7EB830F4FEA830204EB810150
:1017F80024D95FFA82F90823A7EB0907304601F0DC
:1018080057FBFFB209F108034A4903F0FC033A46C3
:10181800304601F04DFB029B08F1030803EB9803E7
:101828000293AB69002B43D12F6954E062689A4256
:1018380091D8A260304607B0BDE8F08308233A4645
:10184800E6E7012B5BD1BDF80C303948C3F38311AF
:10185800062928BF062161F38913023101F00F011F
:101868008900ADF80C3001F0E1FA0646002846D0B0
:1018780001F00BFB0023082203A9304601F018FBF6
:101888000027BDF80C20C2F38312BB00974203F176
:101898000803C6D202994A1CC1F309010331029216
:1018A80004EB81010422304601F002FB0137E8E72E
:1018B800304601F0EEFAFFF733FF80F00100C6B2C0
:1018C800B8E7FB685B7923B13B6831461B6838464B
:1018D8009847FB681F68002FF3D1304601F0D9FA0A
:1018E8000DF107008DF8077000F040FBAB690BB9EC
:1018F800029BA3609DF8070000F068FBDBE72C69FA
:1019080054B90D4B0D480E49C01AC008000440F0E8
:10191800020000F073F8CEE7236820469B689847DA
:10192800E3681C68ECE7002684E700BFE45A00205F
:1019380030960700F05A0020C0950700C0950700B0
:10194800E89707002DE9F34704460F46914601A999
:10195800012218461E46FFF7FDFDDFF89C8078B38C
:10196800019D0023A81CB34203EB000132D11E489D
:10197800002100F01DFC80F3100A1C4B1C4A4FEAA2
:1019880014499B1AB9EBD30F04D31A4940F2A91092
:1019980000F058FB6B1CC3F30903E40008EB830356
:1019A80004F0380449EA0A40C5F3090544F0010483
:1019B800D860033544EA861343EA872348F825307C
:1019C80098F800301BB1FFF7B5FE0028FBD102B034
:1019D800BDE8F087C1F3090108EB810159F823201C
:1019E800CA600133BFE700BF006B002030960700D4
:1019F800C095070062970700E45A002000231A46A2
:101A0800FFF7A0BF07B50123019201AAFFF79AFFCC
:101A180003B05DF804FB07B5CDE9002302236A464D
:101A2800FFF790FF03B05DF804FB1FB5CDE9012374
:101A3800069B039301AA0323FFF784FF05B05DF813
:101A480004FB1FB5CDE90023069B0293079B039374
:101A58006A460423FFF776FF05B05DF804FB7FB5FF
:101A6800CDE90123089B0393099B04930A9B0593E3
:101A780001AA0523FFF766FF07B05DF804FB000025
:101A88002DE9F7430446D01C8846164601A90022D2
:101A98008008FFF75FFD254D98B3019FB81C0190A2
:101AA800C0F30900C0F58063B6EB830F00F10300B3
:101AB8004FEA830905EB80002CD83246414607F0EF
:101AC800C3FC1B48002100F073FB80F310007B1C53
:101AD800C3F30903C7F30907220C05EB8303033794
:101AE80042EA0040E400D86004F0380455F8273092
:101AF80044F0020444EA865203F47C131A4345F87E
:101B080027202B781BB1FFF715FE0028FBD103B067
:101B1800BDE8F0834A46414607F096FCA6EB090269
:101B280008EB090105F10C00C9E700BFE45A0020E1
:101B3800006B002030B50E4C226903460020114688
:101B480029B9D968087142B923610A6030BDC968EA
:101B58000D79854206D00968F2E7D26814680C60EE
:101B68001360F3E701300A28E9D14FF0FF30EDE7C1
:101B7800E46A002038B5084B03F580520125146942
:101B88001D7004B938BDE3685D71236820465B6841
:101B98009847E3681C68F4E7E45A002030B5C38826
:101BA80085B004460D4633B1144A00921449154ACB
:101BB800284600F001FC217A05291DD0637A4BB133
:101BC800A088FFF797FD104B104953F820202846AE
:101BD80000F0F2FB227A0E4BA08853F822200392E1
:101BE8000021FFF76BFD039A0A490346284605B012
:101BF800BDE8304000F0E0BB05B030BD2C980700D0
:101C0800149807000C9807009C9807005DC8070007
:101C1800C09807003198070007B503460846197AA7
:101C2800052911D05B7A2BB1094A0A49019000F0C5
:101C3800C3FB01980849019000F0BEFB019803B06E
:101C48005DF804EB00F0A6BB002AF8D0F2E700BF6D
:101C58002C9807005DC80700299807002DE9F04374
:101C680085B01F460C9D002395F80C902B730646F3
:101C78000C46904629463846FFF790FFB8F1060F04
:101C880009D8DFE808F00412181F2833400031464D
:101C9800284600F091FB002229463846FFF7BCFF92
:101CA80085F80C9005B0BDE8F083226831462846D7
:101CB80000F082FBEFE7D4E900233146284600F024
:101CC8007BFBE8E7A36800933146D4E90023284664
:101CD80000F072FBDFE7E3680193A36800933146E5
:101CE800D4E90023284600F067FBD4E72369029370
:101CF800E3680193A36800933146D4E9002328469A
:101D080000F05AFBC7E76369039323690293E3680A
:101D18000193A36800933146D4E90023284600F0D4
:101D28004BFBB8E708292DE9F74F80460E461746C2
:101D38001C463DD800251B7B257321461046019380
:101D4800FFF72CFFDFF88CA0DFF88CB0AE4232D959
:101D580018F805205946204600F02EFB0135082DBD
:101D6800F4D11B49DFF874A0DFF874B0204600F006
:101D780023FB4FF000094E4524D918F809507E2D51
:101D88001ED8284607F024FB002814BF2A462E2216
:101D98005946204600F010FB09F10109B9F1080F76
:101DA800E9D1012221463846FFF736FF019B23730C
:101DB80003B0BDE8F08F5146204600F0FDFACDE7AC
:101DC8002E22E5E75146204600F0F6FAE4E700BF88
:101DD80045980700419807003B980700439807007B
:101DE800479807004B1C30B5DB00044612F003008F
:101DF8009BB20DD1074D2A601A44074B1A60074B56
:101E08001870074B1870074B1C80074B198030BDA2
:101E18000720FCE7A46B0020A06B00209C6B00202F
:101E2800AC6B0020A86B0020AA6B00202DE9F743BB
:101E3800DFF8BC80B8F800308B4206460D461746DE
:101E480047D300240DF107008DF8074000F08EF805
:101E5800224B234A23481B78008892F800C0844507
:101E68005FFA8CF138BF4C1CDBB238BFE4B2A34236
:101E780028D014781178CBB2884286BF0133DBB200
:101E8800002313709DF8070000F0A0F84FF6FF73C9
:101E98009C4220D0144B1B6843F8347003EBC409F0
:101EA8009EB195B1114BB8F800001B682A4631461F
:101EB80004FB003007F0C8FAA9F80450002003B06A
:101EC800BDE8F0834FF6FF74DCE70020A9F80400B2
:101ED800F5E70920F3E70420F1E700BFAC6B002029
:101EE8009C6B0020AA6B0020A46B0020A06B002034
:101EF800A86B002070B5104C104D22782B789A42B0
:101F080000D170BD0E480F4A2378126806880E4823
:101F180002EBC301006852F83320898803FB0600EE
:101F280090470A4922780988D3B2914286BF013383
:101F3800DBB200232370E0E7AC6B00209C6B002031
:101F4800A86B0020A46B0020A06B0020AA6B0020C7
:101F5800EFF30583C3F308032BB9EFF31480C043F1
:101F680000F00100704701207047000070B504467A
:101F7800FFF7EEFF012803D01049432000F062F874
:101F8800EFF3108672B60E4A9068012398B99360F1
:101F98000C4B0D4DD3F8801029401160C3F88050C8
:101FA800D3F8841051604FF0FF32C3F884202070BA
:101FB80006B962B670BD2370FAE700BFD49807006F
:101FC800B06B002000E100E0FC06FFBD10B5044640
:101FD800FFF7BEFF012803D00949512000F032F86D
:101FE800084B9A685AB154B9EFF3108172B6064A91
:101FF80018681060586850609C6001B962B610BDDE
:10200800D4980700B06B002000E100E030B53AB189
:102018001368DB430A4D0144814204D1D84330BDE3
:102028004FF0FF33F6E710F8012B5340082213F066
:10203800010418BF2C46013A84EA5303F7D1EBE7B1
:102048002083B8ED07B5CDE900016A46002144F2C6
:10205800020002F0DDF803B05DF804FB10B561B1D1
:10206800B2FBF3F403FB1424A4B244B9C0E900148E
:1020780084608281C381204610BD0E20FCE70920C0
:10208800FAE782B050E8022FC188B2EB324F4FF026
:10209800000317BF92B241EA014142EA014104E05C
:1020A8004268B2EB324F08BF012340E80212002A0F
:1020B800E8D18DF807309DF80730002B0CBF1120B0
:1020C800002002B0704737B550E8013F9DB2C4897F
:1020D80025448489A54228BF2D1B0489A54202BF37
:1020E800BFF32F8F002207E0C5EA030540E801543B
:1020F800002CE9D14FF001028DF803200193019AD9
:102108000A609DF8031001F0FF0321B1006810FA7E
:1021180082F003B030BD1846FBE70A884B889A4224
:1021280009D150E8012FC2EA024240E80123002BFE
:10213800F7D1012070470020704737B550E8023FBB
:102148001FFAA3F5C488A54202BFBFF32F8F002250
:102158000DE0C48925448489A54228BF2D1BC3EA04
:10216800054540E80254002CE8D14FF001028DF8F3
:1021780003200193019A0A609DF8031001F0FF0300
:1021880021B1006800EB124003B030BD1846FBE7F0
:102198000A884B889A4209D150E8022FC2EA2242A3
:1021A80040E80223002BF7D1012070470020704738
:1021B80010B5034653E8000F0A4643E8002494F09C
:1021C800000FF7D110BD10B5034653E8000F40EAE1
:1021D800010243E8002494F0000FF6D110BD10B5B9
:1021E800034653E8002F42EA010043E8000494F054
:1021F800000FF6D110BD10B5034653E8000F00EAF2
:10220800010243E8002494F0000FF6D110BD10B588
:10221800034653E8002F02EA010043E8000494F063
:10222800000FF6D110BD10B5034653E8002F02EB9E
:10223800010043E8000494F0000FF6D110BD10B57A
:10224800034653E8002FA2EB010043E8000494F092
:10225800000FF6D110BD0121FFF7B5BF0121FFF72F
:10226800BEBF0021FFF7C7BF0021FFF7D0BF0000A6
:1022780010B50446002834D003681BB91A49FF205A
:10228800FFF7E0FE636823B917494FF48070FFF742
:10229800D9FEA36823B9144940F20110FFF7D2FE12
:1022A800E36823B910494FF48170FFF7CBFE238A06
:1022B80023B90D4940F20310FFF7C4FED4E9012306
:1022C80021689B1ADBB20A60013BDBB2FF2B226854
:1022D80002D10020107110BD1168481C10600B70ED
:1022E800F2E70E20F7E700BF6199070037B504460B
:1022F80020B913494FF49270FFF7A4FE00250DF1A1
:1023080007008DF80750FFF731FE226863681168EF
:1023180099420ED9481E106011F8013CE568218ADF
:1023280001FB0355A36811791B1ADBB2994238BF28
:1023380013719DF80700FFF749FE284603B030BD2A
:102348006199070037B50C46054620B9104940F297
:102358004710FFF777FE24B90D494FF4A470FFF733
:1023680071FE00230DF107008DF80730FFF7FEFD21
:102378002A681368591C1160E968641A298AB4FB31
:10238800F1F41C709DF80700FFF720FE03B030BD84
:102398006199070010B5044618B906493120FFF7BE
:1023A80051FEA2682AB16369216820699847002311
:1023B800A36010BDE09907000EB433B5059D04462F
:1023C80018B911494220FFF73DFE63691BB90E4950
:1023D8004320FFF737FE23681BB90B494420FFF75A
:1023E80031FE63681BB908494520FFF72BFE35B15C
:1023F80006AB01AA29462046019300F079F802B0FD
:10240800BDE8304003B07047E09907000A2938B5A5
:1024180004460D4602D10D21FFF7F8FFA368226894
:10242800591CA160D554D4E901329A4204D32046FC
:10243800BDE83840FFF7AEBF38BD00002DE9F84FC2
:102448009846DDE90A43154682460F460A464FF08C
:102458000109AA420FD2C14538BFC14613F0010B8A
:1024680001D16CB900240126B8F1010F1BD908F17C
:10247800FF386E43F8E709F10109B2FBF5F2E8E726
:102488009B070ED5B8F1000F0CBF30262026A145BA
:10249800E9D2013C31465046FFF7B8FF002CF6D18F
:1024A800E0E72026F3E7B7FBF6F39D42E1D9DFF832
:1024B8003C80B7FBF6F3504618F8031006FB137779
:1024C800FFF7A4FF3346AB42B6FBF5F6F1D2BBF1FA
:1024D800000F02D00CB1A14501D3BDE8F88F20212F
:1024E8005046013CFFF792FFF4E700BFD19A07007E
:1024F8002DE9F74F88461746054620B9AF4940F2FF
:102508005220FFF79FFD6B6923B9AC494FF4157052
:10251800FFF798FD2B6823B9A84940F25520FFF72B
:1025280091FD6B6823B9A54940F25620FFF78AFD53
:10253800B8F1000F00F03E8118F8011B49B92B7B58
:10254800002B00F03781284603B0BDE8F04FFFF7B5
:1025580021BF252940F0B780002698F800302D2BA0
:10256800424608F1010823D0302B24D02B2B25D04C
:1025780000242A2B02F1010123D13B681A1D1B6894
:102588003A601C440A4613782E2B26D101324FF0AC
:10259800000A104610F8011BA1F1300CBCF1090F1C
:1025A8001DD80A2303FB0A13A3F1300A0246F0E7F9
:1025B80046F00106D1E746F00206CEE746F00406EB
:1025C800CBE711F8013CA3F130000928DBD80A2237
:1025D80002FB0434303C0A46CBE74FF0000A12F8FD
:1025E800011B01F0FB0068289046F8D0782909D82B
:1025F8006F290CD8632962D022D8252963D058299D
:1026080000F0888098F80030002B95D197E7703952
:102618000829F7D801A353F821F000BF972707002E
:102628000D2607000D2607002D2707000D26070099
:102638000B2707000D2607000D2607001D2707009A
:10264800642901D06929DDD13A68D2F80090111DBA
:1026580089EAE9723960A2EBE9724FF0010B092AA5
:1026680035DCD34538BFD3462CB1B9F1000F01DBB7
:10267800720700D5013CB30702D5BAF1000F03D0A9
:10268800F00701D44CBB0024B9F1000F2DDAC9F1D1
:1026980000092D212846FFF7B9FE06F00302022A99
:1026A80004D1BAF1000F01D11CBB0024CDE90046CA
:1026B80053460A2249462846FFF7C0FEA2E73B6870
:1026C8001A1D19783A602846FFF7A0FE9AE70A23F0
:1026D8000BF1010BB2FBF3F2C1E7A345D4D22021E1
:1026E8002846013CFFF792FECCE77107D5D52B2190
:1026F800D0E7A345DAD230212846013CFFF786FE11
:10270800D2E73968CDE900460A1D3A6053460A22E5
:102718000968D0E739680A1D3A60CDE90046534692
:102728001022F5E73B681A1D3A6016F00106D3F847
:10273800009024D1B9F1000F03D0484606F002FFFB
:102748000646B4421DD809F1FF3919F8011F0029BE
:102758003FF458AF2846FFF759FEF6E728460136FA
:10276800FFF754FE19F806100029F7D1A642BFF466
:1027780049AF20212846013CFFF748FEF6E700262E
:10278800F0E720212846013CFFF740FED9E73B68E7
:102798001A1D3A60302128461C68FFF737FE782159
:1027A8002846FFF733FE00220823CDE900322146F0
:1027B800102280E703B0BDE8F08F00BF559A0700EC
:1027C80070B50D461646044618B908495520FFF756
:1027D80039FC1DB905495620FFF734FC2B682560E4
:1027E80031462046BDE87040184700BFE19A07000F
:1027F8002DE9F041DDF818800E4617461D460446BF
:1028080018B922498820FFF71DFC1FB91F498920E4
:10281800FFF718FC23681BB91C498A20FFF712FC34
:1028280045BB1A498B20FFF70DFCB20703D01749A7
:102838009120FFF707FCBB0703D014499220FFF74C
:1028480001FCE3689E4204D322696B1E3344934221
:1028580003D90E499320FFF7F5FB2368CDF81880BC
:10286800D3F80CE03A462B4631462046F446BDE8FC
:10287800F041604763685A68B5FBF2F302FB1353F3
:10288800002BD2D001498E20CDE700BFE19A070086
:102898002DE9F0410D4616461F46044618B9194958
:1028A8009E20FFF7CFFB23681BB916499F20FFF72F
:1028B800C9FB1EB91349A020FFF7C4FB63681B6856
:1028C800013B2B4203D00F49A320FFF7BBFBE36872
:1028D8009D4207D363681A686B1E02FB06332269A0
:1028E800934203D90749A520FFF7ACFB2368D3F827
:1028F80010E032463B4629462046F446BDE8F04102
:10290800604700BFE19A070070B550B90E4D0F4CF3
:102918000026641B1423B4FBF3F4B44208D100204E
:1029280010E00368002BF1D0BDE87040DB69184760
:102938002B6813B901361435EFE7DB692846984749
:102948000028F7D070BD00BF685900207C590020CE
:10295800014B436000207047749B0700084670478E
:1029680000207047024B1868003818BF01207047D4
:10297800BC6B002008B50248FFF776FC002008BDB4
:10298800BC6B002008B510461A4606F05DFD002015
:1029980008BD00002DE9F041804686B011480F4679
:1029A80016461D46FFF757FC0446C8B9AA08314623
:1029B800384600F0B3FC0B48FFF756FCD8F808304F
:1029C80053B101228DF800200C9A0592CDE90147F8
:1029D800CDE9036568469847204606B0BDE8F08112
:1029E8001124F9E7BC6B00202DE9F043814687B03C
:1029F80014480E4615469846FFF72DFC0446F0B9D4
:102A08000746BD4215D10F48FFF72EFCD9F808300C
:102A18005BB102228DF800200022CDE90126CDE924
:102A28000325CDF8148068469847204607B0BDE8CE
:102A3800F08306EB073000F043FC0137E1E711248F
:102A4800F3E700BFBC6B002029DF704728DF704721
:102A580070B503689E6886B004460D466EB11422B0
:102A68000021684606F019FDA368059323790195AE
:102A78002BB1012B0DD06846B04706B070BD0123BD
:102A88008DF8003023690293E36803936369049324
:102A9800F1E702238DF80030E3681B030293F5E7A2
:102AA8000846704700207047024B187A003818BF54
:102AB80001207047AC6D0020034B187A0122B0FA50
:102AC80080F05A7440097047AC6D002008B5104674
:102AD8001A4606F0B9FC002008BD000008B514220B
:102AE8000021044806F0D9FC0348FFF7CAFA002081
:102AF80008BD00BFAC6D00209C6D002010B5094CCE
:102B0800094B43602046FFF7A6FB48B906F07CFA5C
:102B1800064920741C2306484FF4EE72FFF79EFA0C
:102B2800002010BDAC6D0020A09B0700C06B0020EA
:102B38009C6D002038B5224D224C2B7A3BB9224996
:102B48002248FFF7FAFA206008B9686038BD022306
:102B580024682B72237973B1012B22D020460321DC
:102B6800FFF776FF00232B726B6017491748BDE803
:102B78003840FFF70DBBD4E90523D21A142AD4E94B
:102B8800031028BF14229208012A38BF01221944D1
:102B98001844FFF759FF50B11128DFD101232B72D8
:102BA800D4E7D4E903031844FFF750FFF3E72B7C7D
:102BB800002BCBD1BDE83840022000F009B800BF97
:102BC800AC6D0020C46D0020C06D00209C6D0020FD
:102BD80038B5224C237A002B3FD0022B09D1032889
:102BE8002ED01F4B00221B68E2601A793AB1012AE5
:102BF80020D0637C6BBBBDE83840FFF79BBFD3E9AF
:102C080005128D1A142D94BF521914329A619142EB
:102C1800EFD102284FF0000308BF19462372104B6A
:102C280018BF0D211868FFF713FF0E490E48FFF76C
:102C3800AFFADEE71A6901321A615B699A42E7E77F
:102C4800E3680133082B01D8E360D2E70023E3608F
:102C5800DFE7BDE8384006F0C7B938BDAC6D0020E5
:102C6800C46D0020C06D00209C6D0020831E012BC8
:102C780001D8FFF7ADBF704700F0FD03012B08D165
:102C8800044B00225A74421E504250411874FFF7F8
:102C980051BF7047AC6D002010B5064C201DFFF7E2
:102CA800DAFA28B9637C1BB9BDE81040FFF742BFC8
:102CB80010BD00BFAC6D00202DE9F34180460D46E4
:102CC800104801A916461F46FFF7FDF90446B0B1A2
:102CD80018220021043006F0E0FB2D0B012323719C
:102CE80001A90848C4F80080A760E5606661FFF79D
:102CF80014FAFFF7D1FF002002B0BDE8F0810420EC
:102D0800FAE700BF9C6D00202DE9F34180460F468D
:102D18000F4801A916461D46FFF7D5F90446A8B184
:102D280018220021043006F0B8FB089BA36001A913
:102D3800C4E903670648C4F800806561FFF7EDF948
:102D4800FFF7AAFF002002B0BDE8F0810420FAE7EF
:102D58009C6D00202DE9F74F99469DF8303000937F
:102D680088469346064618B92349B620FFF76AF9FC
:102D7800F28871794A43043A4A4505D81E490192B6
:102D8800C420FFF75FF9019ADBF80070B6F806A0D7
:102D980007EB0901914209F1040488BFA2EB090776
:102DA800B4FBFAF5CBF800700AFB154445B9AAEB59
:102DB800040BBB4528BFBB462FB903B0BDE8F08F55
:102DC8003668013DF2E7009B043408EB0500344403
:102DD8005A466BB12146A7EB0B0706F035FBBA45FF
:102DE8005D443668D3464FF0000428BFBB46E3E78E
:102DF80001462046EFE700BFCC9B0700FFF738BA33
:102E0800F8B546790146721E0546002393422D689F
:102E180003D30024A64202D8F8BD0133F6E70F68B1
:102E28002846FFF78FFA01343946F3E72DE9F843CE
:102E3800068ACD1C0746FFF759FA043E3544044676
:102E4800B5FBF6F5F0B14FF48073EDB28380C68020
:102E5800013D076081464FF00008A84512D2384668
:102E6800FFF744FA064648B163790133637108F104
:102E78000108C9F8000007608146EEE72046FFF721
:102E8800BFFF34462046BDE8F88301210430FFF730
:102E9800CAB910B5012104460430FFF7D0F9C0B211
:102EA80020B92046BDE81040FFF7AABF10BD0000BA
:102EB8001FB5144603920022009203AAFFF74AFFA7
:102EC800039BA34203D00349F620FFF7BBF804B0E5
:102ED80010BD00BFCC9B07001FB51446039201220A
:102EE800009203AAFFF736FF039BA34204D00349CD
:102EF8004FF48070FFF7A6F804B010BDCC9B070014
:102F0800836800225A60C3E904229A60DA601A6072
:102F18007047000038B50D46044618B909495020D5
:102F2800FFF790F81DB907495120FFF78BF82B6878
:102F38006A686360934208BF0023256008BF636026
:102F480038BD00BF4B9C070010B5044618B90B49A3
:102F58006320FFF777F823681BB908496420FFF757
:102F680071F8636843B12268916852680B449342D0
:102F7800636004BF0023636010BD00BF4B9C070063
:102F880010B50D49A1F59472914201D800200FE0C7
:102F98008C1AE30F03EBE4035B1002EBC30452F853
:102FA8003330834205D802D204F10802ECE76068A6
:102FB80010BD2146E8E700BFD8A1070008B5FFF714
:102FC800DFFF024B002808BF184608BD9DA0070078
:102FD8002DE9F04FC9B008AA01F1400514464B7815
:102FE8000E781B0443EA0663CE7833438E780431A7
:102FF80043EA06238D4244F8043BF0D11024916B38
:1030080016464FEAF14383EA714383EA9123716AD2
:10301800366852F8045F31440B444FEAB54181EAFF
:10302800F51181EAD50101340B44402CD363E6D174
:10303800D0E914E30093836D0193C36D0293036E8B
:103048000393436E0493836E0593C36E0693DDE981
:10305800057BDDE9031CDDE901592B4B009E079335
:1030680074464FF00008079B53F8042B07934FEA68
:10307800F12383EAB11383EA716A08AB53F8283065
:103088001A440AEB020327EA010A01EA0C028AEA57
:1030980002021A444FEA743A86EA05035A44234066
:1030A8008AEAB40A06EA050B83EA0B0B8AEAB45AE1
:1030B80008F10108DA44B8F1400F02EB0903BB46F6
:1030C8005244A94619D172440265009A22444265C5
:1030D800019A32448265029A2A44C265039A1A44C4
:1030E800049B02660B444366059B63448366069B08
:1030F8003B44C36649B0BDE8F08F674635468C4609
:10310800264619461446AEE7D8A1070030B5E0B107
:103118000F4A104900240025C0E91245C0E91412DD
:103128000D4C0E4A0E4DC0E916420E4AC0E918521F
:103138000D4A826602F17452A2F523020023A2F618
:1031480092420364C266184630BD0E20FCE700BFF9
:1031580085AE67BB67E6096A72F36E3C3AF54FA520
:103168007F520E518C68059BABD9831F70B5F0B1A7
:10317800DAB900201CE00C468D180026AC42F8D0C5
:10318800036C14F8012BC2540133402B0364F5D1AE
:103198000146FFF71DFFD0E9123213F5007342F123
:1031A8000002C0E912320664E8E70029E3D10E20E4
:1031B80070BD70B50D4616460446002876D0002925
:1031C80074D0036C8022591C372BE25408443FD832
:1031D800C3F13702002106F060F9D4E91223216C0B
:1031E8000820E1FB0023C4E9122312BAE26323FAA0
:1031F80000F284F83B3084F83A201A0C1B0E214662
:1032080084F8392084F838302046FFF7E1FE691E3B
:103218006EB30023E26EDA4001F8012FA26EDA40A5
:103228000A71626EDA400A72226EDA400A73E26D3F
:10323800DA400A74A26DDA400A75626DDA400A76DD
:10324800226DDA400833202B0A77E3D1002070BDC5
:103258004029C3F13F024FF0000188BF002206F069
:103268001CF921462046FFF7B3FE3822B2E718239F
:10327800226DDA4001F8012F626DDA400A71A26D01
:10328800DA400A72E26DDA400A73226EDA400A7492
:10329800626EDA400A75A26EDA400A76E26EDA40A9
:1032A800083B13F1080F0A77E2D1CFE70E20CEE7EB
:1032B800024AD2F80034002BFBD0704700E00140EE
:1032C8000A4908B50223C1F80435BFF36F8FBFF36D
:1032D8004F8FC1F80805FFF7EBFF0023C1F804354D
:1032E800BFF36F8FBFF34F8F08BD00BF00E00140F1
:1032F80010B5094C0123C4F80435BFF36F8FBFF331
:103308004F8F0160FFF7D4FF0023C4F80435BFF3E3
:103318006F8FBFF34F8F10BD00E0014070B50E4EA8
:1033280001231546C6F80435BFF36F8FBFF34F8FDF
:103338000024AC4207D10023C6F80435BFF36F8FD1
:10334800BFF34F8F70BD51F8243040F82430FFF799
:10335800AFFF0134EDE700BF00E0014043689B6820
:10336800184708B5436808305A7900F0F1FE002084
:1033780008BD2DE9F0410C469CB008461F46039253
:10338800FFF7ECFFD4F80480039998F80550BD4284
:1033980028BF3D4606462A4604A800F0BDFE98F818
:1033A800052022990CA800F0D3FE00960CAB2A4603
:1033B80004A904F1080001F005FE002848F2425073
:1033C80018BF00201CB0BDE8F0810023C0E902321C
:1033D8008B881A44B1F9063002611A44C0E9001119
:1033E80042610888003818BF012070474268118878
:1033F80038B50346002937D0148A02F1100141601C
:103408002CB9C2680168FFF7E0FF204638BD907804
:10341800118900F03005302D14D1947C04F030046B
:10342800302C1BD190881969091A19610021908ADA
:10343800B2F9162008441969014419611144596107
:103448000120E3E700F0F004202C07D15089414324
:10345800002DECD1986801309860E8E700F0C000D2
:10346800802808BF0421F3E70846CFE770B546680F
:1034780004460D4663681A88AA4204D19B7803F073
:103488000F03082B07D12046FFF7B0FF6368B3424C
:10349800F0D1002070BD0120FCE743681A44426067
:1034A80011B101399A4201D10120704713F8010B7B
:1034B80001F8010FF6E770B54568AA7802F00F0623
:1034C800082E86B003461FD103691C6800260CB974
:1034D80006B070BD236862689D68267329466846F1
:1034E800FFF773FF6368049304F10C030593AB784B
:1034F80003F0C003802B08BF231D684608BF049350
:10350800FFF7D9FFA468E2E712F0C00122D102F068
:10351800300010280CD15A691170072EEC68186910
:103528000BD10146204606B0BDE8704000F01AB83D
:103538009006F2D55B691980CAE72A89214624B129
:1035480006B0BDE8704005F07FBF06B0BDE870402A
:1035580005F0A3BF8029BBD1006900219206016054
:10356800B6D5E7E77FB50A4601466846FFF72DFF5F
:1035780030B16846FFF79FFF6846FFF737FFF7E768
:1035880007B05DF804FB836810B504460BB900204A
:1035980010BD0368012298470028F8D0A368013BB2
:1035A800A360F5E72DE9F3410F460DF107018046C9
:1035B800FFF7E9FF054620B90025284602B0BDE817
:1035C800F0819DF907309DF80740002B13DA04F0CD
:1035D8007F0407260DF107014046FFF7D4FF0028B6
:1035E800EAD09DF8072002F07F03B3401C4313067E
:1035F80006F1070601D43C60DFE7232EEAD1DBE7BA
:1036080030B5044685B01546A9B90268114B9A42EF
:1036180011D0102D06D82A4669462046FFF7F0FF3C
:1036280005B030BD102269462046FFF7E9FF0028A3
:10363800F6D0103DEDE7A368AB4201D20020EFE7DA
:1036480023682A46204698470028F7D0A268521BCC
:10365800A260E5E7A3340700F7B50E4601A90746BF
:103668001546FFF79FFFA0B1019A511C4FF00004C7
:1036780004D2B37803F0C003802B01D1204608E0C0
:1036880033898B42FAD329463846FFF7B9FF019BA5
:10369800EC5403B0F0BD73B50D4601A906461446B7
:1036A800FFF780FF98B1019AB2F5803F11D2AB784D
:1036B80003F0C003802B02F102010AD02B898B4250
:1036C80007D32146304621F8022BFFF799FF02B0B5
:1036D80070BD0020FBE7000010B5034C826000229B
:1036E800C0E90041C26010BDA33407002DE9F341D1
:1036F800002580460E462F462C460DF10701404610
:10370800FFF741FFC0B19DF807C0A4F120030CF0FA
:103718007F02C4F1200102FA03F322FA01F10B43FC
:10372800A2401CF0800F45EA020547EA030704F1AE
:10373800070404D1C6E9005702B0BDE8F081462C61
:10374800DBD10020F8E737B50D4669461446FFF788
:10375800CDFF70B12B89082B0DD1DDE90032C4E90A
:103768000032DDE90001914208BF98420CBF0120F8
:10377800002003B030BD042B03D1009B236000223E
:10378800EFE7022B03D1009B23809BB2F7E7012BC5
:1037980004D1009B237003F0FF03F0E70020E8E763
:1037A80037B50D4669461446FFF7A0FF30B12B899F
:1037B800082BDDE9001203D1C4E9001203B030BDC3
:1037C800042B4FEAE17009D121600B460246824280
:1037D80008BF8B420CBF01200020EFE7022B03D16A
:1037E8000BB22380DA17F2E7012B02D14BB2237018
:1037F800F8E70020E2E7F7B51F4600233B700D46C7
:103808000B70136001A904461646FFF7CBFE30B9CA
:10381800A36813B901233B70002003B0F0BD019CDD
:10382800002CF7D0E30804F0070433602C70F4E7A9
:1038380013B50446052925D8DFE801F0030F17243E
:103848002422012201A92046FFF7DAFE18B19DF9CA
:103858000430002BF5DB02B010BD08220021204601
:1038680002B0BDE81040FFF7CBBE01A9FFF79AFEF2
:103878000028F0D0019A00212046FFF7C1FEEAE7B0
:103888000422EBE70020E6E773B50D4601A90446DC
:10389800FFF788FE064618B90026304602B070BD0C
:1038A80094E80F0085E80F0001998A42F4D3A960D3
:1038B800A3685B1AA360F0E72DE9F0435668B37874
:1038C80013F0C00489B007468C46154603D0402C37
:1038D80069D000240CE003F00F02604903F03003C4
:1038E800202B51F8228025D006D8E3B1102B17D011
:1038F800204609B0BDE8F083302BF9D16B693188D7
:103908001980072A09D121463289286905F0C5FDA1
:103918006B682969D868FFF725FE2A69696840E05D
:103928006B6901221A702A693146434609B0BDE81D
:10393800F0431847BCF1020FD5F8149024D1042A9B
:1039480022D804A9FFF7A0FF04460028C1D0069B8F
:103958002BB16968B9F800304A899A4205D8059BA5
:103968007B60069B002BC3D0B3E708892A6903FB59
:10397800002204A8C04728B1B9F800300133A9F8DB
:103988000030E4E70446EAE7B9F8003072899A4261
:103998009FD931892A69581C03FB0122A9F8000024
:1039A80031463846C1E7D2F81080464656F8043BFF
:1039B80023B909B0BDE8F043FFF73ABF022914D193
:1039C80004A9FFF761FF002883D0D8F800306968A0
:1039D800324604A89847044600283FF47AAF069B6D
:1039E800002BF2D1059B7B6082E7012926D00529AF
:1039F8002CD000297FF46DAF0C460DF10409013479
:103A08000B2C3FF466AF012249463846FFF7F8FD14
:103A180000283FF45EAF19F9013B002BEFDB104B98
:103A2800049301ABCDE90534002307936968D8F8FE
:103A38000030324604A89847044659E7082201A9ED
:103A4800FFF7DEFD08240028E9D142E704220DEB48
:103A58000201FFF7D5FD0424F5E700BFE4A2070043
:103A6800A33407002DE9F04F91B00446002604A8BE
:103A7800CDE90266FFF7A9FCA3683BBBDDE9053485
:103A880004A89D78FFF7B2FC0028F7D115F0300F95
:103A980003D1059B1B8803B10134002C00F0A980D9
:103AA800630902A90022934240F09C8010AA02EB0D
:103AB800830304F01F0453F8383CC4F120044FF08A
:103AC800FF30E040C31A584258410DE00DF103039E
:103AD80001AA0DF102012046FFF78DFE38B99DF8C5
:103AE8000330002BCAD1002011B0BDE8F08F019936
:103AF80004A8FFF7BBFC002850D1019BB3427DD33B
:103B0800059D059A937803F00F03082B7FD004A82E
:103B1800FFF76CFC059B9D42F3D14FF0FF36019FE8
:103B2800B7426BD3089B9DF802A0D4F808801D68A3
:103B38004FF00109A368002D5DD098459CD12B68F2
:103B4800D3F800B0BBF1000F08D053463A462946D7
:103B58002046D8470028C6D0AD68EBE7D3F808B0B0
:103B6800BBF800309F42F7D16A6859460AA8FFF7A8
:103B78002CFC6B680E9305F10C030F939BF8023035
:103B880003F0C003802B04BF2B1D0E930AAA85F8EF
:103B98000C9051462046FFF78FFEDBE7059B9B788C
:103BA80013F0300F0FD1069A3F2A0CD8510910ABE9
:103BB80003EB810102F01F020123934051F8382CD6
:103BC800134341F8383CE5682DB19DF8022001996E
:103BD80004AB2046A8479DF8021004AA2046FFF728
:103BE8006BFE10E051F8045B01357FF47DAF0132C4
:103BF80059E7012078E798457FF43EAF9DF8021019
:103C08002046FFF715FE00287FF436AF6BE71688CD
:103C180085E737B50C460546114620460192FFF761
:103C2800A1FC019A2146284603B0BDE83040FFF7C1
:103C380019BF70B586B0CE6801920C4602A9054638
:103C4800FFF722FE68B1E06858B1A378019A03F043
:103C58003003202B314602A805D1FFF7DAFF039B7A
:103C68006B6006B070BDFFF7FDFEF8E713B50C46B4
:103C78006946FFF73BFD60B1DDE900134A0842EAF7
:103C8800C372C9074FEA530344BFD243DB43C4E9B5
:103C9800002302B010BD37B50D4669461446FFF73C
:103CA800E5FF70B12B89082B0DD1DDE90032C4E99D
:103CB8000032DDE90001914208BF98420CBF0120A3
:103CC800002003B030BD042B03D1009B2360DA171A
:103CD800EFE7022B03D1BDF900302380F7E7012B72
:103CE80003D19DF900302370F1E70020E9E713B50F
:103CF80004220C460DEB0201FFF782FC08B1019B80
:103D0800236002B010BD1146FFF7F1BF13B50822BA
:103D18000C466946FFF774FC18B1DDE90023C4E9D5
:103D2800002302B010BD1146FFF7F0BF08B54309E4
:103D38000CBF4FF0FF33002300F01F0023FA00F000
:103D4800C30704D403494FF4F670FEF77BF94FF02C
:103D5800A04008BD08A30700032810B5044603D9EE
:103D680006494120FEF76EF9054B1C5D2046FFF71A
:103D7800DDFF0123A340C0F80C3510BD33A30700B5
:103D8800A4A30700032810B5044603D90649472011
:103D9800FEF758F9054B1C5D2046FFF7C7FF0123C6
:103DA800A340C0F8083510BD33A30700A4A307003B
:103DB80008B50020FFF7E6FF0120FFF7E3FF022028
:103DC800FFF7E0FFBDE808400320FFF7DBBFC207AD
:103DD80038B5044616D51120FFF7A8FF0325C0F80B
:103DE80044571220FFF7A2FFC0F848571320FFF7E7
:103DF8009DFFC0F84C571420FFF798FFC0F85057A4
:103E0800FFF7D6FFA30714D50D20FFF78FFF0C246B
:103E1800C0F834470E20FFF789FFC0F838470F2055
:103E2800FFF784FFC0F83C471020FFF77FFFC0F87A
:103E3800404738BD38B1054B0360054B436001234B
:103E48000372002070470E20704700BF833E0700B2
:103E58005D3E070069B10B78022B0CD1022804D013
:103E6800032814BF08201120704703230B7000207B
:103E780070470E2070470820704710B50C4681B176
:103E88000B78012B06D00ED9033B012B94BF0820D9
:103E9800112010BD03F0FEFE0028FAD10223237082
:103EA800F7E70E20F5E70820F3E7000070B5144B9C
:103EB800144A0C21D21AB2FBF1F2816911F8025CA2
:103EC800044635B900690021914205D101232360D8
:103ED8000EE04FF0FF30F6E71E68AE420CD1461CEC
:103EE80007D19D68D4E90001D4E90223A8472060DE
:103EF80070BD5E688642F4D001310C33E4E700BF40
:103F0800B4950700C09507001EF0040F0CBFEFF32F
:103F18000880EFF30980FFF7C9BF00BF28B139B1A6
:103F28000023C1E900301846704748F21050704726
:103F380048F21350704730B1036848F240508B4242
:103F480008BF0020704748F21050704728B148F267
:103F58001150914208BF0020704748F21050704736
:103F680070B506460C461D46FFF7D8FF50B9B37921
:103F78004AB1AB420AD111462046FFF7F2F908B917
:103F8800044B236070BD48F21050FBE748F2115013
:103F9800F8E700BF7052464D2DE9F0470C4606463B
:103FA8000F492046DDE9088915461F46FFF7C3FF7C
:103FB800A0B963685A79494652004046FFF7C6FFE0
:103FC80060B94DB1CDF820803B462A46214630469F
:103FD800BDE8F047FFF7CDB948F21050BDE8F087CB
:103FE8007052464D10B5044638B149B10B6841606E
:103FF800984708B9044B236010BD48F20150FBE70D
:1040080048F21050F8E700BF6E524648F0B4134625
:1040180048B10768094EB7420AD161B12AB143686D
:10402800F0BC5B68184748F201531846F0BC70476B
:1040380048F20253F9E748F21053F6E76E52464841
:10404800F0B460B107680C4EB7420CD171B1436847
:104058001568DC68A5420CD3F0BC9B68184748F289
:104068000150F0BC704748F20250FAE748F213508A
:10407800F7E748F21450F4E76E524648F7B504469D
:10408800DDE9086715460193FFF7ACFF68B9019AA7
:1040980029462046FFF7BAFF38B93A463146204646
:1040A80003B0BDE8F040FFF7CBBF03B0F0BD0000A0
:1040B800F8B50A4F0A4C0B4EE41B0123E408337091
:1040C8000025A54203D1022333700020F8BD57F81C
:1040D800353098470028F9D10135F2E7AC9507004B
:1040E800AC950700C86D002038B50D46044618B9D0
:1040F80008493320FDF7A6FF691E21442046814266
:1041080000D238BD03780A7800F8012B01F801398C
:10411800F5E700BFA8A3070070B50D46144606468C
:1041280018B90A494520FDF78DFF1DB907494620F2
:10413800FDF788FF621E3244013DB24200D270BDD5
:1041480015F8013F02F80139F7E700BFA8A30700F7
:1041580070B5164604460D46FFF7DEFF3246A9192C
:10416800A019BDE87040FFF7D7BF38B50D46044623
:10417800FFF7BAFF29466019BDE83840FFF7B4BF1A
:1041880008B507281BD8DFE800F004121A1A1A0429
:104198001A040120FFF71BFE0020FFF7DDFD0120B8
:1041A800FFF7DAFDBDE808400220FFF7EBBD01206C
:1041B800FFF7E8FDBDE808400220FFF7CDBD08BDC8
:1041C80008B5FDF7D7FCFDF7B5FA0028FBD10D4D72
:1041D800642445F001054FF47A40A847013CFAD120
:1041E800094BD3F8F020D20700D500BEBFF34F8F9C
:1041F800D968064A01F4E0610A43DA60BFF34F8FD9
:1042080000BFFDE700A5070000ED00E00400FA0587
:1042180007B50B46064C07490092641AE4082404C3
:104228000246054944F00100FDF7FFFBFFF7C8FF10
:10423800C0950700C095070070A4070008B502469E
:10424800054B064806491B1ADB081B0443F001000E
:10425800FDF7D8FBFFF7B4FFC0950700C09507002E
:10426800A7A4070010B501F011FF4FF480510020FA
:1042780001F0DDFA08B1FFF7E1FF1548C0F5FC21B0
:1042880001F0D5FA01460028F5D11248124CFDF785
:1042980001FAFDF729F9114B1149E41AE40824043D
:1042A80044F00300FDF7AAFB0E4801F061F900286D
:1042B800E1D1FDF73FFA0028FBD10B4944F001009A
:1042C800FDF79CFBFDF736FA0028FBD1D3E700BFCA
:1042D80000100700B95B0700C0950700C0950700EC
:1042E800C2A4070089410700CEA407008B18104418
:1042F8008B4200D1704713F8012D00F8012DF7E724
:104308000000000000000000C3F10803DB0070B5E6
:1043180001330446002003A55B1920C940CAAD1922
:1043280020C4184720C940CA754120C420C940CAC2
:10433800754120C420C940CA754120C420C940CA5B
:10434800754120C420C940CA754120C420C940CA4B
:10435800754120C420C940CA754120C4404170BD80
:104368000000000000000000C3F10803DB0070B586
:104378000133002403A500BF5B1920C940CAAD1B47
:1043880020C0184720C940CAB54120C020C940CA2A
:10439800B54120C020C940CAB54120C020C940CA83
:1043A800B54120C020C940CAB54120C020C940CA73
:1043B800B54120C020C940CAB54120C06441B4FA03
:1043C80084F0400970BD00BF2DE9F04F08B4F8CA69
:1043D80004B451F8042BA3FB028940F8048B4FF076
:1043E800000AE4FB629A4FF0000BE5FB62AB4FF06A
:1043F800000CE6FB62BC4FF0000EE7FB62CE51F802
:10440800042B4FF00008E3FB628940F8048BE4FBBF
:10441800629AE5FB62ABE6FB62BCE7FB62CE51F851
:10442800042B4FF00008E3FB628940F8048BE4FB9F
:10443800629AE5FB62ABE6FB62BCE7FB62CE51F831
:10444800042B4FF00008E3FB628940F8048BE4FB7F
:10445800629AE5FB62ABE6FB62BCE7FB62CE51F811
:10446800042B4FF00008E3FB628940F8048BE4FB5F
:10447800629AE5FB62ABE6FB62BCE7FB62CE40F802
:10448800049B40F804AB40F804BB40F804CB40F868
:1044980004EB0CBC052B00F01E810C68A0F1140085
:1044A800A1F11401A2F1140252F804EB4FF0000537
:1044B80050F8046BE4FB6E5652F804EB50F8047B9A
:1044C800E4FB6E6752F804EB50F8048BE4FB6E785B
:1044D80052F804EB50F8049BE4FB6E8952F804EBA5
:1044E80050F804ABE4FB6E9AA0F1140052F8044BA8
:1044F80051F804EB4FF0000CE4FB6EC540F804CB18
:1045080051F804EBE4FB6E5640F8045B51F804EBF9
:10451800E4FB6E6740F8046B51F804EBE4FB6E783B
:1045280040F8047B51F804EBE4FB6E8940F8048BF7
:1045380051F804EBE4FB6E9AA0E80006062B00F0A5
:10454800CA800C68A0F11800A1F11801A2F11802A4
:1045580052F804EB4FF0000550F8046BE4FB6E567C
:1045680052F804EB50F8047BE4FB6E6752F804EB56
:1045780050F8048BE4FB6E7852F804EB50F8049B77
:10458800E4FB6E8952F804EB50F804ABE4FB6E9A36
:1045980052F804EB50F804BBE4FB6EABA0F1180032
:1045A80052F8044B51F804EB4FF0000CE4FB6EC5D5
:1045B80040F804CB51F804EBE4FB6E5640F8045B7A
:1045C80051F804EBE4FB6E6740F8046B51F804EB18
:1045D800E4FB6E7840F8047B51F804EBE4FB6E8949
:1045E80040F8048B51F804EBE4FB6E9A40F8049B06
:1045F80051F804EBE4FB6EABA0E8000C072B6AD083
:1046080008B40C68A0F11C00A1F11C01A2F11C0265
:1046180052F804EB4FF0000550F8046BE4FB6E56BB
:1046280052F804EB50F8047BE4FB6E6752F804EB95
:1046380050F8048BE4FB6E7852F804EB50F8049BB6
:10464800E4FB6E8952F804EB50F804ABE4FB6E9A75
:1046580052F804EB50F804BBE4FB6EAB52F804EBE1
:1046680050F804CBE4FB6EBCA0F11C0052F8044BDC
:1046780051F804EB4FF00003E4FB6E3540F8043BBF
:1046880051F804EBE4FB6E5640F8045B51F804EB78
:10469800E4FB6E6740F8046B51F804EBE4FB6E78BA
:1046A80040F8047B51F804EBE4FB6E8940F8048B76
:1046B80051F804EBE4FB6E9A40F8049B51F804EBC4
:1046C800E4FB6EAB40F804AB51F804EBE4FB6EBCC2
:1046D800A0E8001808BCBDE8F08F002310B51C4600
:1046E8005AB2914200DC10BD40F823400133F7E78D
:1046F80010B500231A465CB2A14203DCB2FA82F07C
:10470800400910BD50F8234001332243F3E74A1112
:10471800012350F8220001F01F0103FA01F10840BB
:104728007047013910B549B2041D0A06CBB204D44A
:10473800013954F82120002AF7D001335BB273B154
:1047480003F18042013A50F82220002022B9013BAF
:1047580000EB431318B210BD52080130F6E71846B3
:10476800F9E710B500235CB2A24200DC10BD51F895
:10477800234040F823400133F5E710B5013A52B21F
:10478800130601D5002010BD50F8224051F8223000
:104798009C4205D802F1FF32F2D24FF0FF30F2E727
:1047A8000120F0E700EB81010023884200D3704725
:1047B80051F8042D43EA52030B60D307F5E737B5E8
:1047C8001D469DF9183001930446FFF79DFD019B96
:1047D80038B91A4621462846FFF7CFFF0128019B22
:1047E80007D02A462146204603B0BDE83040FFF7EF
:1047F800BBBD03B030BD37B51D469DF918300193D8
:104808000446FFF7B1FD019B38B12A4621462046F0
:1048180003B0BDE83040FFF777BD03B030BD2DE9E8
:10482800F04FB5B004AC9DF9F8501F4680462B46B2
:104838002046FFF7C9FD24AB29463846CDE90234A6
:10484800FFF76FFFC0EB851004B2002C2146B8BFFC
:1048580004F11F01634203F01F0341F3471104F001
:104868001F0614A858BF5E42FFF737FF002E08B294
:104878002BDD14AB002203EB8000C6F1200E13469B
:10488800AB4217D36B00019314AB03EB85096F1E82
:1048980034AB012603EB8707002C54DA34AB03EB67
:1048A80086062A4656F8C81C4046FFF75AFF35B018
:1048B800BDE8F08F57F823C00CFA06F10A4340F818
:1048C800042B01332CFA0EF2DAE714AB2A463946E8
:1048D80003EB8000FFF745FFD4E70FFA82FE5AF892
:1048E800C83C53F82EB034AB03EB8202013052F8C7
:1048F800803C0B44BBEB030334BF012200229B45E1
:1049080018BF11465CF8C82C42F82E30019B42B201
:104918009A42E2DB731A5E42294614A85E41FFF709
:1049280041FF34AB03EB8503294653F8802C57F835
:10493800803C43EAC27347F8803C4846013CFFF795
:1049480031FF24B2A8E734AB0020C6F1010C0146C0
:1049580003EB860A03EB8C0CD8E730B51C4691B004
:10496800054693F900306846FFF72EFDD4F8AC30C1
:1049780069462846984711B030BD13460A46FFF7E6
:10498800ECBF2DE9F04793F9006092B004468946E0
:104998001046314615461F46FFF7AAFE002840F08C
:1049A80091803A46494602A8FFF7E7FF3B4602AA2C
:1049B80021460AA8FFF7D1FF02A908463A46FFF7A1
:1049C800DCFF3B462A4649464846FFF7C6FF07F143
:1049D80004083A4629462846FFF7CFFF43462A46A9
:1049E800214620460096FFF7EAFE43462A46294616
:1049F80028460096FFF7E3FE43462A462146284606
:104A08000096FFF7F8FE3B462A4621462046FFF768
:104A1800A4FF43462246214628460096FFF7CFFECC
:104A2800434600962A4621462046FFF7C8FE2368DB
:104A3800DB074AD53346424621462046FFF764FC49
:104A4800314682462046FFF7ADFE06F18043013B22
:104A580054F8232042EACA7244F823203A462146F1
:104A68002846FFF78AFF43460AAA294628460096A1
:104A7800FFF7C1FE43460AAA294628460096FFF7D3
:104A8800BAFE0AA9084643462A460096FFF7B3FE2F
:104A98003B460AAA21462046FFF75FFF02AA434683
:104AA800104621460096FFF7A6FE324629462046C4
:104AB800FFF757FE49462846FFF753FE02A9484626
:104AC800FFF74FFE12B0BDE8F08731462046FFF7EA
:104AD80069FEC3E72DE9F04115468AB004460E4643
:104AE8001C22002103A804F0D8FC2F1D95F9008092
:104AF80003232A46314620460293FFF73EFF3B46F2
:104B080002AA21462046CDF80080FFF774FE2B4606
:104B1800324621462046FFF720FFCDF800803B466D
:104B280005F1840221462046FFF749FE0AB0BDE898
:104B3800F08100002DE9F042082288B0FFF711FE4D
:104B4800CB6A03930B6B04934B6B05938B6B0693A8
:104B5800CB6B07930C4681460027134669466A4685
:104B68006846CDE901770097FFF7CEFB0823054695
:104B78006A4649464846FFF7C7FB236B0393636BB6
:104B88000493A36B0593E36B0544CDE906376A46A6
:104B9800082369466846FFF7B7FB082305446A46B9
:104BA80049464846FFF7B0FB236A0093636A0193BE
:104BB800A36A0293A36B0693E36B07930544082348
:104BC8006A4649464846CDE904770397FFF79CFBB8
:104BD800636A0093A36AA26B0193E36A0293049247
:104BE800636BE26B0393CDE90523236A07932E18C1
:104BF80008236A4649464846FFF786FBE36A00935E
:104C0800236B0193636B0293236A0693A36A07934A
:104C1800351808236A4649464846CDE9047703977C
:104C2800FFF7A2FB236B0093636B0193A36B0293C3
:104C3800E36B0393636A0693E36A07932E1A0823C8
:104C48006A4649464846CDE90477FFF78DFB636B12
:104C58000093A36B0193E36B0293236A0393636A44
:104C68000493A36ACDE90537236B0793361A082303
:104C78006A4649464846FFF777FBA36B0093E36B08
:104C8800CDE90137636A0393A36A0493E36ACDE924
:104C98000537636B0793361A08236A464946484620
:104CA800FFF762FB361A0E4C0FD436B90822494674
:104CB8002046FFF762FD01280FD008232246494607
:104CC8004846FFF751FB361AEFE7082322464946C4
:104CD8004846FFF719FB3618F7D408B0BDE8F0824C
:104CE8000CA5070070B514468AB006460D461A464C
:104CF800214602A80193FFF740FE019B02AA314614
:104D08003046FFF72AFE02A9019B22460846FFF714
:104D180024FE019B02AA29462846FFF71EFE0AB078
:104D280070BD2DE9F0478AB01446DDF848A0554615
:104D38001F4615F9046B0096804689462B460246A5
:104D4800214602A8FFF757FD02A952460846FFF779
:104D580014FE534602AA41464046FFF7FEFD53465D
:104D680002AA21462046FFF7F8FD2B464A46394657
:104D780038460096FFF73FFD5246394602A8FFF72E
:104D8800FCFD02A92B46424608460096FFF733FD74
:104D980002A92B46224608460096FFF72CFD2B4613
:104DA8004246214620460096FFF725FD53462246F7
:104DB80049464846FFF7D1FD2B4602AA4146204600
:104DC8000096FFF718FD5346224639463846FFF746
:104DD800C4FD2B464A46394638460096FFF70BFD78
:104DE800324602A92046FFF7BCFC0AB0BDE8F087AE
:104DF8002DE9F0471F46B3F9023013F11F0448BFED
:104E080003F13E04DD1D48BF03F10E056611EC10E9
:104E1800944275B228BF144689462946FFF75DFCBF
:104E2800224649468046FFF761FAB7F90230B3EBEC
:104E3800C40F4FEAC4021FD2D21A08EB860400211D
:104E4800C2F12006A0450ED324372A4641463846EB
:104E5800FFF793FC01280FD02B463A464046BDE8A1
:104E6800F047FFF781BA54F8040D20FA02F30B4318
:104E7800236000FA06F1E5E7BDE8F08770B503683E
:104E880013F001060546144605D013460A460146A6
:104E9800FFF73AFA064621462846FFF783FC46B153
:104EA80004F18042013A55F8223043F0004345F8B6
:104EB800223070BDF0B50F46A1B0064619463846F7
:104EC80015461C46FFF714FC28B1304621B0BDE852
:104ED800F040FFF702BC224639466846FFF741FC1E
:104EE800294608A8FFF73DFC10A82146FFF7F5FB67
:104EF800012318A81093FFF7F0FB224608A968467B
:104F0800FFF73BFC30B9224610A93046FFF729FCD1
:104F180021B0F0BD009BDA0709D421466846FFF7A7
:104F280041FC2246294610A8FFF7A8FFE5E7089BA1
:104F3800DB0707D4214608A8FFF734FC2246294698
:104F480018A8F1E7002823461CDD08AA6946684628
:104F5800FFF70AFA21466846FFF724FC224618A9FB
:104F680010A8FFF70AFC002805DA10A923462A46EC
:104F78000846FFF7C9F910A9234618AA0846FFF7FB
:104F8800F3F9CEE76A4608A8FFF7EEF9214608A824
:104F9800FFF708FC224610A918A8FFF7EEFB002827
:104FA80005DA18A923462A460846FFF7ADF918A9D5
:104FB800234610AA0846FFF7D7F9BFE7004870470D
:104FC80008A507002DE9F04F2DED028BEBB00D463B
:104FD800769E03901946B6F9023096F9004013F10F
:104FE8001F0848BF03F13E0848F3471808F1FF3B84
:104FF80022AB002743F82B706AAB03EB8B034AA85C
:1050080043F8807C43F8607C924696F90120FFF7CC
:105018006DF996F9012052A81144FFF767F9214666
:105028004AA8FFF765FB8146002840F0278152A86F
:10503800FFF75EFB0290002840F0228106F1240968
:1050480042464AA94846FFF798FB012840F01A81D2
:10505800424652A94846FFF790FB0128049040F0C9
:1050680011810AAF43464A461AA8FFF723FF029B5D
:1050780047F82B305246294638463346FFF7B8FEE4
:10508800394638464B461AAACDF80080FFF7C7FBC9
:105098005AAD4B461AAA4AA912A8CDF80080FFF7C4
:1050A800BEFB224628460399FFF75BFBA300059346
:1050B800039B05EB840A03EB840106F1440B50467D
:1050C800FFF74FFB594632A8FFF74BFBA3000BEB4A
:1050D80003013AA8FFF745FB331D294632AA1AA84F
:1050E800009408EE103AFFF786FB53462A463AA981
:1050F80032A80096FFF715FE1AA9084618EE102ADE
:105108002346FFF7D7FE1AAA514628463346FFF72B
:10511800E9FD029BCDE9063B039B41463846CDE9B4
:105128000835FFF7FEFA4146834612A8FFF7F9FA59
:105138005845B8BF584685B2691E09B2384603912A
:10514800FFF7E5FA0399071E12A818BF0127FFF712
:10515800DEFA002814BF022000200DF1180A0743C8
:1051680022465AF8271022A8FFF7FBFA0DF1A80BE0
:10517800A30019445846FFF7F4FA1AA82146FFF786
:10518800ACFA049B0360023D22AB2DB20393824626
:10519800002D26DA18EE102A234651465046FFF70E
:1051A80089FE0398334652465946FFF79BFD0399FB
:1051B80042464846FFF7E1FA012804D043464A46EA
:1051C8000846FFF7D1F8013C64B24AAA23064AD53B
:1051D800029BB3FA83F040096BB0BDEC028BBDE8CB
:1051E800F08F33465246D6F8A47003985946B8470C
:1051F80029460AA8FFF78BFA2946071E12A818BFE6
:105208000127FFF784FA002814BF02200020074373
:1052180006AB53F8271019B3224632A8FFF7A1FAB4
:10522800059B3AA81944FFF79CFA014633465246B3
:1052380032A8FFF757FD18EE103A0399009432AAE6
:1052480042A8FFF7D8FA039A00965B463AA932A813
:10525800FFF767FD334642AA51465046FFF77DFBEC
:10526800013D2DB294E7039B52F8241053F82430E3
:105278004B40029919430291013CA7E73846ABE736
:105288004846A9E70298A7E70369C26893429CBF0A
:1052980080681B18013B981A70472DE9F843D0E93C
:1052A80002940546A9EB04084068904520440F463F
:1052B800144404D904F0C8F8EC60BDE8F883424609
:1052C800A4EB090404F0C0F86868224607EB08015B
:1052D800F0E72DE9F843C5680646894617464FF0BA
:1052E80000083469B3687068A54228BFE418013C17
:1052F800621B5C1BBC4228BF3C46944228BF144634
:1053080049462844224604F09FF8B3682544AB4236
:1053180008BF00253F1BA044A144F560E1D14046E9
:10532800BDE8F88310B5114C114AA2610223C4E903
:105338000433104BE361A2644FF480530E4A0F49C3
:105348002362E26400231022E01DA3626362E36229
:10535800A3656365E365226504F0D2F80849204631
:1053680004F0CEF82023A37110BD00BFCC6D00203F
:10537800B8A50700546E0020446E0020C1A50700A0
:10538800C5A5070070B5164B182400FB04451D443D
:1053980004FB00331646DC6A012C0ED0022C18D010
:1053A800E4B92846FFF770FF864204D832462846FB
:1053B800FFF773FF3446204670BD2846FFF764FFA9
:1053C8008642344628BF044622462846FFF765FF32
:1053D800F1E72846BDE87040FFF77BBF0024EAE705
:1053E800CC6D0020FFF79EBF41DF70476DDF70472F
:1053F800014B01221A7070477482002008B5FCF72F
:10540800B9FBFCF797F90028FBD1BFF34F8F05498B
:10541800054BCA6802F4E0621343CB60BFF34F8FB9
:1054280000BFFDE700ED00E00400FA0508B50948F3
:10543800094B0A49C01AC008000440F00400FCF7F0
:10544800DDFA074B074800221A70BDE8084002F051
:10545800C7BB00BFC0950700C0950700CCA50700D3
:10546800748200200554070008B50748074B08490F
:10547800C01AC008000440F00300FCF7BFFABDE8FA
:105488000840FFF7D3BF00BFC0950700C0950700CD
:10549800E2A50700042810B5044609D802280DD84B
:1054A80012D00B4B1B6893B12046BDE8104018473B
:1054B800831F012BF5D8FFF7B9FFF2E705494FF431
:1054C800701000F035FBECE702F07EFAE9E710BD5A
:1054D800788200207154070008B543090CBF4FF0CB
:1054E800FF33002300F01F0023FA00F0C30704D4A1
:1054F80003494FF4F670FCF7A5FD4FF0A04008BD36
:1055080008A3070008B50648064B0749C01AC00893
:10551800000440F00400FCF771FA002008BD00BF49
:10552800C0950700C0950700F6A507001FB502A89B
:10553800FFF75CFF08B1FEF781FE0A4B0A489DF8A9
:105548000C200A49C01AC0089DF80E3000930004C8
:105558009DF80D3040F00300FCF767FA05B05DF8E0
:1055680004FB00BFC0950700C095070010A6070000
:10557800F8B5754B754C7649E41AE408240444F0F0
:10558800040605463046FCF739FA724B10201D60B8
:10559800FFF7A2FF704BC0F84037002002F036FB3F
:1055A800002879D100F07CFC01286ED0022875D043
:1055B800002871D14FF08043D3F8005415F480359A
:1055C80015D04FF48032C3F800240546634F3B6A78
:1055D800012B1FD0624944F00300FCF70FFA614920
:1055E8003046FCF70BFA01254FF4701759E0D3F851
:1055F800202502F0F802A82A0AD1D3F82025D007DE
:1056080006D5D3F8202502F05602C3F82025DDE799
:105618000125DBE74FF440535A68534B9A420FD1A8
:105628007A6B1DB997F86032012B09D04F484FF4B7
:10563800805103F045F918B94D4944F00200CCE710
:1056480002F00AFCBA6901461DB997F8A132012B8C
:1056580005D0484803F034F908B94749EDE7474908
:105668003046FCF7CBF91020FFF736FFD0F810359D
:10567800D90301D44249B3E74FF08043D3F81C550E
:1056880015F0B105B0D03F49AAE7FFF7CFFE3E4974
:1056980044F00100FCF7B2F90320F8BD01254FF4EE
:1056A800A0273A493046FCF7A9F9002D39D000F077
:1056B8004BFD374A20211820FCF794FB08B1FEF770
:1056C800BDFD4FF08043D3F81C2502F0F802B02A44
:1056D80009D1D3F81C25D20742BFD3F81C2502F004
:1056E8004E02C3F81C25FFF70DFF0028D4D1384619
:1056F800284900F01DFA284800F004FF0028CBD103
:1057080026493046FCF77AF9FFF710FF00F062FDF2
:10571800FCF7F0FBFCF70EF80028F7D1FFF764FE62
:10572800F4E702F0F3FA0028B6D11D4E1D48357093
:1057380002F056FA337823B91B4940F22F20FCF7C0
:1057480081FC00F033F8A2E7C0950700C095070078
:1057580032A60700788200200C000300489A002037
:1057680049A60700E7A60700DBE5B151A89C002081
:1057780077A60700E99C0020B2A60700DAA6070072
:105788000AA7070029A707004AA7070056A7070086
:10579800547E0020715407009D54070064A7070039
:1057A80074820020F953070074A7070037B5184B17
:1057B800184C194D1949E41AE408240444F004006B
:1057C8004FF480520190FCF71DF9D5F88020144958
:1057D8000198FCF717F94FF0FF33C5F88030C5F88A
:1057E8008031C5F88430C5F8843101F0A5FD20B1B9
:1057F8000C4944F00100FCF701F9FBF79BFF002876
:10580800FBD14FF4805003B0BDE8304000F03CB805
:10581800C0950700C095070000E100E0FBA707005E
:1058280031A807005BA8070080F30888084770B50F
:10583800C1F30B0434BBB0F5FE2F23D84B1E1B0B52
:10584800020B03EB103101264FF08040914201D248
:10585800204670BD02F01F03550906FA03F3032D15
:1058680005D8DFE805F00206090CC0F80036013259
:10587800ECE7C0F80436FAE7C0F81036F7E7C0F8E6
:105888001436F4E70724E3E738B504462648C0F59C
:10589800FE21FFF7CCFF054668B12448244B254973
:1058A8001B1ADB081B0443F001002A46FCF7AAF880
:1058B8002846FEF7C3FC02F0CFFA1F4B9B6903F69C
:1058C800FF7323F47F6323F00F0319180020FFF7F9
:1058D800AEFF054668B11548154B18491B1ADB0879
:1058E8001B0443F001002A46FCF78CF82846FEF713
:1058F800A5FCEFF305820023D4E9005483F3148850
:1059080083F3108883F3118883F31388C2F30802A2
:105918001AB10B495820FCF795FB21462846BDE8EB
:105928003840FFF781BF00BF00100700C09507008F
:10593800C095070090A80700489A0020C7A807004C
:10594800FBA8070073B5274B064627481B1ADB0838
:105958001B040C463246254943F00400FCF752F874
:10596800B4F1807F39D322498F20FCF76BFB6FF0AD
:105978007F41A14228BF21461E4B641AD3F8045523
:10598800631E942B96BF9634746074600D44347B08
:1059980025F07F4598BF963D032C03D914497720FD
:1059A800FCF750FB134E04F5A8734FF4F86046F863
:1059B8002350114B43F001039847104BA2001344A6
:1059C80000221A601B680193019B4FF4803303FA8D
:1059D80004F4C6F8044302B070BD952CC7D8044936
:1059E8009020C2E7C0950700C095070092A907005C
:1059F800A8A907000040024060AA070040410240F1
:105A08001FB518490B7853BB4FF08043A024D3F837
:105A18001824D2035CBF01229A60134B0022C3F8FA
:105A28000021D3F8000103900398C3F84021D3F86C
:105A3800400102900298C3F84421D3F84401019030
:105A480001980A4880F82443102444600220C3F8CF
:105A5800082501229A601A60C3F804030A7004B08A
:105A680010BD00BF808200200040024000E100E03D
:105A7800264B2DE9F743D3F8042152B124490A688B
:105A880001320A600022C3F80421D3F804310093DC
:105A9800009B204D204B214C214EDFF89080DFF8F1
:105AA8006C90204FED1AED082D0445F0040533687D
:105AB800CBB1002333603368019322464146284620
:105AC800019BFBF79FFF227B17494FF480339340DC
:105AD800C9F8083322462846FBF794FF616851B19C
:105AE8002046FFF72FFF0436BE4204F11004DED132
:105AF80003B0BDE8F083A16811B12046FFF722FF8B
:105B08002368002BEFD09847EDE700BF0040024024
:105B18007C820020C0950700C095070084590020AA
:105B280040410240484102404CAA07003AAA0700F7
:105B3800F8B5114B114E0446114837681B1ADB089B
:105B48001B043A4643F004000D460E49FBF75AFF82
:105B58003A7B4FF4803393400B4AC2F808334CB178
:105B68003668FFF74DFF356021463046BDE8F840FE
:105B7800FFF7E8BEF8BD00BFC0950700A459002094
:105B8800C09507003AAA07000040024070B5074BCD
:105B98001D6804460E46A860FFF732FF2E602146B6
:105BA8002846BDE87040FFF7CDBE00BFA8590020C9
:105BB800034A044B1068D3F8043503EB00607047C0
:105BC8007C82002000400240014B01221A7070477D
:105BD800818200202DE9F341264FFB6A7E6ABC6C66
:105BE800AC2B38D17B6B1C44F61A234B234D244A2B
:105BF80024490096ED1AED082D0445F004082346C3
:105C08004046FBF712FFFB6AAC2B06D11C48324614
:105C1800A4F5804103F0E1FB18B319483246214648
:105C280003F0DBFBE8B11849334622464046FBF750
:105C3800F2FEFBF77FFD0028FBD100F0CBFA2046EF
:105C4800314601F05BFB044680B1104945F0010084
:105C5800FBF7D4FE0AE0002CC7D102F011F9044684
:105C6800C3E70B494046FBF7C9FE0024204602B0B3
:105C7800BDE8F081489A0020C0950700C09507004C
:105C88000010070066AA07009BAA0700FFAA0700E2
:105C9800C8AA07002DE9F04F3C4B16463C4A9B1A10
:105CA80087B0DB081B04814205460F46049343F086
:105CB800040B08D137495846FBF7A0FE00242046BC
:105CC80007B0BDE8F08F03D233494F20FCF7BAF98B
:105CD80036B1C5F30B031BB12F495320FCF7B2F9BA
:105CE8007B1BB3F5805F4FEA133403D22A49572050
:105CF800FCF7A8F900F028FA082C28BF082406F6B3
:105D0800FF7923034FEA1939039405930EB93446F2
:105D1800D5E7039B4B453ABFDDF80CA0DDF81480AE
:105D2800CA464FF000025146284628BFB04601F047
:105D38009FFA04460028C2D11849CDF800802B46A6
:105D48003A465846FBF771FE08F10302234622F053
:105D580003023946284601F04DFA04460028AED120
:105D68000F4A136B4344136301F040FFA9EB0A0980
:105D7800A6EB08064544474404460028C6D0049BC1
:105D8800084943F00100FBF739FE98E7C095070082
:105D9800C095070019AB070028AB0700BDAB07008B
:105DA800489A0020DEAB07002DE9F74302F078F8A7
:105DB800314C324BDFF8E4903149D9F84860D9F8D2
:105DC8003080D9F83450E41AE4082404074644F033
:105DD80004000190FBF712FE06F5005301985A687B
:105DE800284B9A4209D0284944F00100FBF706FEE7
:105DF8000325284603B0BDE8F083D9F83030AB421C
:105E08001E4404D12149FBF7F9FD0025F1E7C3B988
:105E18004FF440521178142982BF1D495269B2FBD0
:105E2800F1F206F5005198BF1A4691F800C0BCF18E
:105E3800140F82BF4969164BB1FBF3F31549FBF701
:105E4800EAFDA5EB080202F6FF7222F47F6222F057
:105E58000F02314607EB0800FFF71CFF054628B183
:105E68000D4944F00100FBF7C9FDC2E703B0BDE8E6
:105E7800F04301F0BBBE00BFC0950700C095070006
:105E880017AC0700DBE5B1513CAC070070AC07006C
:105E980040420F0082AC0700ABAC0700489A0020D4
:105EA8002DE9F047624B634D634E6449ED1AED08E6
:105EB8002D0445F004073846FBF7A0FDF36AAA2B2A
:105EC80000F09A800CD8012B22D0A52B00F08880F6
:105ED80045F003005A49FBF791FD0020BDE8F08723
:105EE800AC2BF5D157493846FBF788FD564938465B
:105EF800FBF784FDFFF758FF0446002800F0868072
:105F0800524945F00100FBF779FD4FF0010823E005
:105F18004F493846FBF772FDD6F82490D6F848A0CA
:105F280001F09AFF346B4B4900EB04083846FBF745
:105F380065FD316B5144884514BFA9EB040200226A
:105F48004046FFF7A7FE044670B1434945F00100FB
:105F5800FBF754FD4FF00008F36A4049224645F02C
:105F68000100FBF758FD13E001F076FF2246494691
:105F7800FCF74CF8B26A904280462AD13849384634
:105F8800FBF73CFD0123C6E90783C6F81890A04635
:105F98003448DFF8F49001F055FF0023324889F8BF
:105FA800003001F023FE99F80030044623B92F4948
:105FB80040F2A510FCF746F88CBBB8F1000F35D0BD
:105FC800336A012B32D138462949FBF717FD0220E5
:105FD80084E70346274945F00100FBF71CFDD6E797
:105FE80025493846FBF70AFDFFF7DEFE4FF00108AA
:105FF8000446002CCCD0AFE720493846FBF7FEFC1E
:10600800FFF7E8FD4FF000080446F2E7FFF7E2FD6E
:10601800044608B11A4974E74FF00108B8E745F09B
:1060280001001849FBF7EAFC032057E7012055E770
:10603800C0950700C0950700489A0020C4AC070027
:10604800D0AD070079AD070087AD0700A4AD070004
:10605800E5AC0700EFAC0700ABAC0700E9AD070003
:106068000AAD07006C9A0020D15B070028AB070037
:106078001BAE07001FAD070067AD070070AD070036
:10608800BAAD070077AE07008182002010B5002462
:10609800D4F8F83F013304D1084940F6F870FDF709
:1060A80027F9D4F8FC3F013307D1BDE810404FF47D
:1060B800FC2140F6FC70FDF71BB910BD001007006D
:1060C8000A4AD2F800347BB109480023D2F80815EF
:1060D800D940C90748BF03F5C07103F1010348BFA0
:1060E80042F82100072BF1D1704700BF00000140A2
:1060F8003546526E08B50748074B0849C01AC0080C
:10610800000440F00300FBF779FCBDE80840FFF706
:10611800D7BF00BFD0950700C095070091AE070014
:1061280007B5084B0022C3F80021D3F800310193CA
:10613800019BFBF71FFDFBF7FDFA0028FBD103B01D
:106148005DF804FB0000014037B5194D2B784BBBB7
:1061580018481949194B401AC008D3F800240004FC
:1061680040F0030002B3D3F80445154901902246D4
:10617800FBF748FC40F616529442B8BF1446A4F503
:106188004864FFF79DFF01980E492246FBF73AFC49
:106198000D492046FFF7FAFC0C4B4FF480321A6089
:1061A80001232B7003B030BD0949FBF727FCF7E743
:1061B80082820020D0950700C095070000000140AA
:1061C8009FAE0700B8AE0700FD60070000E100E0E1
:1061D800EAAE0700034BD3F800340BB1FFF770BFEA
:1061E800704700BF000001404FF08053D3F83001E2
:1061F800421C04BF4FF0704393F8E00F831F5842CE
:10620800584170474FF0704393F8E02F062A09D1A0
:10621800D3F8E83FC3F30313033B032B02D8024A26
:10622800D05C70470020704718AF070008B5FFF72B
:10623800DBFF40B14FF080538F4AD3F82433C3F3C8
:106248000423C2F84035FFF7DDFF10B18B4B8C4AB1
:106258005A67FFF7C9FF48B14FF080534FF08042AB
:10626800D3F84432C3F34233C2F83C35FFF7CAFFD0
:1062780030B1844AD2F8FC3023F08073C2F8FC3085
:10628800FFF7B2FF40B14FF080430022C3F80C2162
:10629800C3F81021C3F83825FFF7B4FF20B14FF039
:1062A80080430322C3F8A025FFF7ACFF60B1764B0B
:1062B8000522C3F810260122C3F888260022C3F855
:1062C80018263F22C3F814264FF08053D3F8302104
:1062D800511C09BF4FF07043D3F8343193F8E02FC5
:1062E800D3F8E83F08BFC3F30313062A4DD1033B95
:1062F800032B03D8654AD35C002B46D04FF080525D
:10630800634BD2F80414C3F82015D2F80814C3F864
:106318002415D2F80C14C3F82815D2F81014C3F8B1
:106328002C15D2F81414C3F83015D2F81814C3F881
:106338003415D2F81C14C3F84015D2F82014C3F849
:106348004415D2F82414C3F84815D2F82814C3F811
:106358004C15D2F82C14C3F85015D2F83014C3F8E1
:106368005415D2F83414C3F86015D2F83814C3F8A9
:106378006415D2F83C14C3F86815D2F84014C3F871
:106388006C15D2F84424C3F87025FFF72DFF48B1E7
:106398004FF080534FF08042D3F8583203F04F0348
:1063A800C2F8E43EFFF720FF48B14FF08043D3F82E
:1063B8000024D20744BF6FF00102C3F800244FF055
:1063C8008053D3F83021062A0ED1D3F83431033B59
:1063D800032B02D82F4AD35C33B12F4AD2F83C376B
:1063E80043F48063C2F83C37264AD2F8883043F435
:1063F8007003C2F88830BFF34F8FBFF36F8F4FF031
:106408001023D3F80022002A03DBD3F80432002B30
:106418002EDA224B0122C3F80425D3F80024002ADF
:10642800FBD04FF010221521C2F80012D3F8002437
:10643800002AFBD04FF010231522C3F80422174B73
:10644800D3F80024002AFBD00022C3F80425D3F88F
:106458000024002AFBD0BFF34F8F0A49104BCA68AB
:1064680002F4E0621343CB60BFF34F8F00BFFDE738
:106478000C4B0D4A1A6008BD0030014000C00740AF
:106488000DF0ADBA00ED00E00050004010AF07007D
:1064980000C0004014AF07000010004000E00140B9
:1064A8000400FA05AC5900200090D00313681F2B94
:1064B80010B5144607D900220830FCF77AFE08B94F
:1064C8002023236010BD48F21450FBE70830FCF786
:1064D8004DBE0830FCF71ABE008800F00100704776
:1064E800831F012B10B5044602D8002001F070FC70
:1064F800034B1B681BB12046BDE81040184710BD70
:106508008482002038B5104B104C1860104B11498C
:10651800E41AE408240444F00300FBF76FFA0020AF
:10652800FFF7DEFF0C4801F019FC054620B9BDE86D
:106538003840094801F0BEB90246084944F0010054
:10654800FBF760FA284638BD84820020C095070012
:10655800C0950700E8B00700E9640700FBB0070032
:106568006CDF70476DDF704772DF704773DF70470D
:1065780074DF704775DF704776DF70477ADF7047E2
:106588007CDF70477DDF70477FDF704786DF7047AD
:106598008FDF704790DF7047A8DF7047AADF70472A
:1065A800ADDF7047AEDF7047B0DF7047B1DF7047CF
:1065B800B5DF704762DF704766DF704713DF7047EB
:1065C80010B5094B0949044609481B1ADB081B0486
:1065D800224643F00400FBF715FA21460548BDE8BA
:1065E8001040FBF7AFBE00BFD895070025B10700E4
:1065F800C09507004496070070B518228CB00DEBC3
:106608000200002102F049FF282308932348244B65
:106618002449254CC01AC0080004012540F0040094
:106628008DF818508DF82D50FBF7E8F91623ADF8C2
:1066380006300023CDE90333059302230622237095
:10664800237159230926A27063710322FE23657002
:10665800E270A3710DF10601A0190294ADF80C6067
:10666800FFF790FFB8B9BDF8063026725A19E271E3
:10667800BDF80C200D4C134402A906AA2046ADF81B
:106688000C30FFF771FF30B92078FFF771FF2078E1
:106698002946FFF76BFF0CB070BD00BFD895070007
:1066A800C095070037B1070006930020B0590020B5
:1066B800F0B50388242B8FB0044651D80BB90FB01E
:1066C800F0BD013B232BFAD801A252F823F000BFFA
:1066D800C96A0700C7660700C7660700C7660700DC
:1066E800C7660700C7660700C7660700C7660700D2
:1066F800C7660700C7660700C7660700C7660700C2
:10670800C7660700C7660700C766070099670700DE
:10671800DD6707008169070035690700D96B070045
:10672800C7660700C7660700C7660700C766070091
:10673800C7660700FB6B0700C7660700C766070048
:10674800C7660700C7660700BD690700C766070078
:106758001B6A0700FD690700E96807001769070059
:10676800503B9AB2062AAAD8062BA8D801A252F8FA
:1067780023F000BF0B680700D56A0700FB6B070012
:10678800C7660700C766070091680700436A0700E5
:10679800AF4BB04DB049B14EED1AED082D0445F0A0
:1067A8000400FBF72BF9A3883380AD4B1B680BB1B2
:1067B80001209847AB493088FFF7DCFE02460028E5
:1067C8003FF47DAFA84945F001000FB0BDE8F040A7
:1067D800FBF718B9A14B4FF6FF721A80A34B1B6841
:1067E8005A0704D4FFF708FF08B1FDF727FD9C4BB3
:1067F8001B68002B3FF463AF02200FB0BDE8F040E8
:1068080018479B4FE288BB889A427FF458AF994853
:10681800904DFBF76BFD8E4BED1AED082D040646E7
:1068280038B9954945F002000FB0BDE8F040FBF7D4
:10683800E5B8F4230093238A9049024645F0040002
:10684800FBF7F3F8228A04F11201304602F0FCFD4E
:106858001822002108A802F020FE08238DF8203015
:10686800874B0A93874B0997CDE90B3608A8238AEB
:10687800ADF8343000F0FEFF00283FF420AF7D482B
:106888003146FBF75FFD1AE7E288F62A24D8D31EC3
:106898009B0723D0D31F9BB2013B594201F0030150
:1068A80003F0030302F1FF3458BF4B42E31A9CB2D2
:1068B800674B68487449C01AC0080004234640F072
:1068C8000400FBF7A8F8654B21461888FFF770FE0F
:1068D80000283FF4F4AE88E0F724E9E71446E7E738
:1068E8005B4B5C486949C01AC008000440F00400CA
:1068F800FBF784F80022A08808A9CDE90822FFF751
:1069080049FE00283FF4DBAEFDF798FCD7E6504B74
:10691800504862895E49C01AC008E389000440F003
:1069280004000FB0BDE8F040FBF775B8484B494C80
:1069380058494A4DE41AE408240444F00404204663
:10694800FBF75CF802230893288806AB08AA42F6EE
:1069580005210993FFF724FE08B1FDF76FFCBDF888
:1069680018204D492046FBF74DF8002328881A4681
:106978008521FFF709FEC4E7354B36484749C01A59
:10698800C008000440F004000390FBF737F8628960
:1069980043490398FBF736F8228942490398FBF7E5
:1069A80031F8A28940490398FBF72CF8E2893F495E
:1069B80003980AE7264B274D3D49ED1AED082D04AB
:1069C80045F00400FBF71AF8244B04F10801188875
:1069D800FFF7D0FD044600283FF471AE0246354962
:1069E80045F00100FBF70EF820460FB0BDE8F04077
:1069F800FDF724BC164B17482F49C01AC008237A44
:106A080000930004637AA27A40F00400FBF70DF8C3
:106A180055E60F4B0F482949C01AC008000440F03A
:106A28000400FAF7EBFF0023A0888DF8203008A9AE
:106A38008DF82130FFF7ACFD63E7A379002B7FF4D5
:106A48003EAE064B13211888FFF796FD40E700BFBE
:106A5800C0950700D895070046B10700B259002035
:106A68002C930020B6B6070050B1070028930020E9
:106A7800F2920020449607007EB107009DB10700FE
:106A88003D6D0700C9650700BDB1070003B20700E7
:106A980034B2070072B207009AB20700BDB207000D
:106AA800E4B20700FAB2070010B3070022B30700E8
:106AB80037B3070066B307009BB30700D5B30700D9
:106AC800554B00211888FFF777FD01E7A379002BC4
:106AD8003FF4F5AD022B7FF4F2AD504D2189AA8920
:106AE80091427FF4ECADA27B012A7FF4E8AD4FF42C
:106AF80080320992228A484EADF82820628AADF881
:106B08002A2004F114020B9205AF298A30880893D1
:106B180006AA06930797FFF743FD60B93846FFF7C3
:106B2800DBFC40B940F2FD133088ADF8243008A9E9
:106B3800FFF73AFDC3E5002308A93088ADF82430F3
:106B4800FFF732FD014600287FF4B9AD182208A8E6
:106B580002F0A3FC237D324A8DF82030022B0995E0
:106B68000A9224D0062B10D0012B10D12D4B1A8855
:106B78002D4B1A80637DD4F816200C93012B0D92AF
:106B880005D12A4801F024F901E0637D0C9308A897
:106B980000F070FE00283FF492AD254A254B2649A7
:106BA8009B1ADB081B04024643F001000DE6204B4C
:106BB80020482249C01AC008000440F00400FAF72F
:106BC8001DFF184AB4F815301380174A1380DEE702
:106BD800174B18481A49C01AC008000440F00400AE
:106BE800FAF70CFF0023A0881A461946FFF7CEFCD7
:106BF8006EE60023A0881A461946FFF7D7FC08B1AD
:106C0800FDF71CFB0B480A4B0E49C01AC0080004CC
:106C180040F0040008E600BFB2590020F2920020BC
:106C28003D6D07003093002032930020AC9507009B
:106C3800C0950700D895070010B40700FEB30700F9
:106C480044B407006AB4070070B5204E346814F0E5
:106C5800010432D01E4B984236D01E4B1E4D1F4C9D
:106C68001F49ED1AED082D0445F004052846FAF7EA
:106C7800C5FE22884FF6FF739A4220D0194928464C
:106C8800FAF7BCFE3368208843F00403132133600D
:106C9800FFF772FC044680B9134EC82446F001067B
:106CA8004FF47A40B047013CFAD102F06DF904463E
:106CB80018B90E492846FAF7A1FE204670BD0C4BBC
:106CC8001878FFF755FCF0E70024F6E72893002032
:106CD800AC950700C0950700D8950700B259002069
:106CE8008CB40700A9B40700B0B60700B8B4070011
:106CF800B05900207FB50023CDF80B308DF80F3048
:106D08000A4BADF806109B89ADF8083001238DF8C1
:106D18000A300DF10603CDE90430054B02A91888A5
:106D2800FFF740FC07B05DF804FB00BFF2920020BB
:106D3800B259002030B50D4687B0044620B94649FF
:106D480040F28710FBF77EF925B943494FF4C47028
:106D5800FBF778F900210D2202A8019102F09DFBB2
:106D68002378082B0BD13D4A3D4913880988013BFC
:106D78009BB2138031B32BBB03231180237063783C
:106D880022788DF805206021012B8DF804108DF8EC
:106D9800063019D033493448401AC0080004334932
:106DA80040F00200FAF737FE63780B2B12D100F09F
:106DB8009BFA8DF80700002000F090FA042101A842
:106DC800FFF798FF07B030BD062A05D0082A29D05A
:106DD800032A27D00321F2E7E1688DF80710D4E9E8
:106DE8000123080A8DF80800080C090E8DF80A100E
:106DF800110A8DF80B208DF80C10110C120E8DF85D
:106E08000E201A0A8DF80F308DF810201A0C1B0E60
:106E18008DF80D108DF809008DF811208DF81230BD
:106E28000F21CCE7D4E90123110A8DF807208DF84A
:106E38000810110C120E8DF80A201A0A8DF80B3062
:106E48008DF80C201A0C1B0E8DF809108DF80D20EA
:106E58008DF80E300B21B2E7D1B407003293002031
:106E680030930020C0950700D89507005DB507004E
:106E78002DE9F041054694B020B9404940F24F4011
:106E8800FBF7E0F83E4B4FF6FF721A8001204FF6F1
:106E980059632A4602A98DF80A00ADF80830FFF7B1
:106EA8007BFB0446002865D1364B04AA03F1100782
:106EB800164618685968144603C40833BB4222466C
:106EC800F7D1A91C3046FFF775FB0446002851D1BD
:106ED80001461C220DA802F0E0FA9DF834308DF826
:106EE800044043F004038DF834300223ADF80C302D
:106EF800AB788DF80E3003238DF80630F423CDE9F6
:106F08000A44ADF82C302B464FF0110833F8040B27
:106F18000C9403AF01AE08AA0DA98DF80580089757
:106F28000996FFF73BFB044620BB01461C220DA82F
:106F380002F0B3FA18238DF834300123ADF80C3081
:106F4800AB788DF80E3013238DF806301723CDE972
:106F58000A44ADF82C302B4608AA33F80C0B8DF8F0
:106F680004400DA90C94CDE908768DF80580FFF74B
:106F780015FB0446204614B0BDE8F081D1B40700E3
:106F8800B259002095B60700F0B5514E336813F09A
:106F9800010485B0074640F099804E4B4E4D4F494D
:106FA800ED1AED082D0445F004052846FAF726FDEC
:106FB8004B4B4C481F60FBF75BF9029400F0AFF9AC
:106FC8000446002873D1484A48492846FAF71AFD6A
:106FD8004548FFF7F3FA0446002868D14449284693
:106FE800FAF70CFD01F092FF044600285FD102A8D1
:106FF80002F05EF80446002859D13E492846FAF7BF
:10700800FDFC02A9012002F05DF8044600284ED1DB
:1070180039492846FAF7F2FC02A802F013F90446A7
:10702800002844D100F062FE002843D0334800F025
:107038004DFE336843F002033360112302A88DF834
:107048000430FFF78FFA044688BB9DF8093002A880
:1070580001338DF80930FFF783FA044638BB3368EB
:107068009B072CD5254C2649A369221D2846FAF7EB
:10707800D2FCA269211D92B201A8FFF781FA044649
:10708800A8B92048FFF77AFA044680B91E48FFF7E6
:10709800EFFE044658B9FFF7AFFA044638B933682B
:1070A8001A4943F0010328463360FAF7A7FC204643
:1070B80005B0F0BD16492846FAF7A0FCBDE715490A
:1070C8002846FAF79BFC14490822D4E70024EEE787
:1070D80028930020C0950700D89507008DB50700B4
:1070E8002C9300204496070000100700ACB5070059
:1070F800CCB50700E1B50700F8B507008882002085
:107108002AB60700B6B60700F29200206AB6070052
:1071180010B607004BB6070084B5070030B51A490A
:107128000B6885B004460BB1013B0B601748184A41
:1071380063682578121AD208120442F004008BB949
:107148000B68144A14490093012D08BF0A46A36826
:107158001249FAF76AFC63699BB1E06805B0BDE8BB
:10716800304018470A68029222690192A2680A49C7
:107178000092084A012D08BF0A460949FAF76FFC30
:10718800E9E705B030BD00BF34930020C095070083
:10719800E0950700C4B60700BEB60700CAB60700E8
:1071A800F0B6070008B502460B4B0C481B1ADB0863
:1071B8001B0443F004004AB10949FAF71FFC0949C6
:1071C8000948BDE808400022FBF7FABA0749FAF770
:1071D80015FC0749F4E700BFE0950700C0950700D4
:1071E8002CB70700AC9B07006859002052B707006E
:1071F800809B07002DE9F7439846174C174BDFF89B
:107208006C90E41AE408D9F800302404CDE900238E
:1072180005460B460E4617461149024644F004003F
:10722800FAF70FFC29460F48CDF800803B46324656
:10723800FBF7DEFA054640B9D9F800300133C9F842
:107248000030284603B0BDE8F0830246064944F002
:107258000200FAF7D7FBF4E7E0950700C0950700AE
:107268007AB7070068590020BDB70700349300209B
:107278002DE9F341134B144C144FE41AE4083B680E
:107288000093240405460B460E46904610490246D4
:1072980044F00400FAF7C9FB29460E484346324633
:1072A800FBF7F6FA054630B93B6801333B602846E0
:1072B80002B0BDE8F0810246074944F00200FAF73F
:1072C800A1FBF4E7C0950700E09507003493002080
:1072D800EAB707006859002027B80700014B187063
:1072E8000B20704738930020024B002218781A7040
:1072F800704700BF3893002018DF704730B585B05D
:10730800054610220C466846002102F0C6F8A4087B
:10731800684601950294FFF7EFFF05B030BD1FB531
:107328000023CDE901330393684602230093FFF756
:10733800E3FF05B05DF804FB4FF000534FF48052B3
:107348001A60002070470000084B09480949C01A14
:1073580010B5C008000440F00400FAF74FFB064BD4
:10736800BDE810401B680620184700BFC0950700FD
:10737800E895070062B80700449300200A2803D95B
:107388000B38C0B2FFF7AABF7047000070B50546BA
:1073980086B00020FBF7B8FA0146A0B1274A1821A9
:1073A8002846FAF743FD00283DD0254A254B2649B3
:1073B8009B1ADB081B04024643F0010006B0BDE837
:1073C8007040FAF71FBB1822684602F066F80423DB
:1073D8001C4C8DF800301A4B1C4EE41A1C4B1A6DCD
:1073E8003368E40824049A4244F004041DD119497E
:1073F8002046FAF703FB184B3168186801F06AFC5D
:107408008DF80100FFF7BAFFD5E901138DF80100E7
:1074180068469847114800F0E9FB9DF8012010499B
:107428002046FAF7EFFA06B070BD01238DF8013057
:107438006846D5E901139847EFE700BF9573070041
:10744800C0950700E895070096B807003C93002010
:10745800489A0020BFB807004093002051730700E6
:10746800EEB807002DE9F041836888B0044623B9D7
:10747800974940F2CF20FAF7E5FD1822002102A82B
:1074880002F00BF80123934E8DF80930924B2278C5
:107498008DF80820F61AF6083604531E46F004053F
:1074A8000B2B00F2C581DFE813F02C000C002C0038
:1074B8002C00C3012C00C3012C00C301C301C3016C
:1074C800110086492846FAF799FA07E028468449C0
:1074D800FAF794FA834B07201B6898479DF8092010
:1074E80081492846FAF78EFAD4E9011302A8984789
:1074F8009DF80930012B00F085817A4B05201B6827
:107508007FE1062A794F01D0012A01D122693A7018
:107518003A78012A09D0022A74D0754946F0010048
:10752800FAF76CFA00233B70C6E0072B64D8DFE853
:1075380003F004631443635B631E6E492846FAF73D
:107548005DFA684B03201B689847606901F092F860
:10755800FFF714FF8DF80900C0E767492846FAF7D6
:107568004DFA664BDA6B1B6C03920493B6E72369FA
:1075780023B9574940F21310FAF764FDA38A23B9D7
:1075880053494FF48A70FAF75DFD5D492846FAF7CA
:1075980035FAA18A206901F085F8FFF7EFFE574B0D
:1075A8008DF80900DA6B1B6C0493E3680392002BD7
:1075B80094D02069984791E752492846FAF71EFA6D
:1075C8005149524801F0ECF8FFF7D8FE01288DF830
:1075D800090083D1002000F009FB08B94C4971E784
:1075E8000A238DF8093079E74A492846FAF706FA56
:1075F8004FF400730593B4E735494FF4BC70FAF7BC
:1076080021FD6BE7072B00F20F81DFE813F008007C
:107618000D01CF00DE000D01FE000D0195003E4971
:107628002846FAF7EBF901F06DF830B93B4946F016
:107638000100FAF7E3F90823D3E7626932B9384958
:1076480046F00100FAF7DAF90323CAE7C2F30B039D
:1076580043B12A4B2C495B6D096813448B4201D016
:107668003049EDE7B2F5805F06D92F4946F00100B1
:10767800FAF7C4F90423B4E7204F23497B6D09685E
:10768800D018884206D9009146F001002749FAF738
:10769800CCF9D0E77A64FA6CBA641C4A3B65106886
:1076A8003B63002201211844FFF7E2FD30B1204975
:1076B80046F00100FAF7A2F9052392E7BB6C0093A4
:1076C8003B6D7A6C1B492846FAF7AFF906E700BF0D
:1076D80016B90700E8950700C0950700A6B9070086
:1076E800CAB9070044930020EEB80700B459002037
:1076F80062BD0700E2B907000CBA0700489A0020EB
:1077080030BA070059BA07003C9300204093002084
:1077180084BA0700A9BA0700D3BA0700FABA070063
:107728002FBB070048BB070069BB07008DBB0700DC
:10773800FEBB070015BC070041492846FAF75EF969
:1077480000F0E0FF00283FF476AF3E4FA18AD7E96A
:1077580014329B1A7A6C0B44934201D93A496FE769
:107768003A4A3B6B1268206903EB020807F14802AA
:10777800FAF74CFCE368064623B935494FF4F8702C
:10778800FAF760FCE368A28A21694046FFF732FDF8
:1077980008B1E3680DE7A38A3A6BBE641A443A63FA
:1077A8003A6D049613443B65039397E6254E2949A1
:1077B8002846FAF723F9B36C326D27492846FAF7B9
:1077C8002AF9B36C0493336DEEE728462349FAF798
:1077D80015F91C48D0E91473426CFB1A934205D082
:1077E8001F4946F00100FAF716F924E7836CC364D1
:1077F8000021416447652046FFF7C8FD194B1B6807
:107808000420984708B0BDE8F08117492846FAF7E0
:10781800F5F80C4B4FF480519A6C1B6D0591009153
:107828000492124903934EE7094940F29720E6E68D
:107838000F4946F00300FAF7E5F80223D1E600BF46
:1078480050BC0700489A002076BC070040930020EF
:1078580016B907008DBC0700AEBC0700C4BC070002
:10786800ECBC07004493002010BD070037BD07009B
:1078780082BD0700836810B58BB10A4A1821FAF750
:10788800D5FA044648B10848084B09491B1ADB08D1
:107898001B0443F00200FAF7B1F8204610BD072494
:1078A800FBE700BF6D740700C0950700E895070067
:1078B800A1BD070038B50546C0B10120FFF772FC2D
:1078C800044648B900F0C8FE00F01CFF30B9084B68
:1078D80000201D60FFF702FD204638BD0549064817
:1078E80000F05EFF0128F2D00324F5E70724F3E750
:1078F800449300203C930020409300202DE9F74357
:1079080017464FF4607298461F4D0646894601F0A7
:1079180064FD1E4BED1AED0804462D0445F00400E5
:1079280054B91B49FAF76AF81FB9002003B0BDE83B
:10793800F0832046B847F8E716490190FAF75EF851
:10794800154901983246FAF75DF8002201213046C0
:10795800FFF78EFC30B1114945F00100FAF74EF8F7
:107968000320E3E74FF460724946404601F06CFD9E
:107978003B464FF4607241463046FFF73BFC002817
:10798800D3D00749E8E700BFF0950700C095070086
:10799800D1BD07001BBE07002FBE07004FBE070062
:1079A80072BE07000368013310B5044609D00022EF
:1079B80058210430FAF72AFB23681B1A5842584109
:1079C80010BD0020FCE700002DE9F0474C48DFF827
:1079D8005C814C4CDFF858914B4EFFF7E3FFD8F829
:1079E80000A007465046FFF7DDFF0546002871D086
:1079F800DAF80450012D0AD00022C3210AF51870C4
:107A0800FAF704FBDAF85C522B1A5D425D41002F4D
:107A180050D0A4EB0907FF083F0447F004073B498F
:107A28003846F9F7EBFF364937484FF4607201F0F2
:107A38000BFD8DB136493846F9F7E0FFD8F800500C
:107A480034485422291D01F0FFFC33484FF43272A8
:107A580005F15C0101F0F8FC7768012F4DD1A4EB2A
:107A68000900C0082D4C2E49000440F00300A4F57D
:107A7800E475F9F7C3FF0FCD0FC40FCD0FC40FCDB9
:107A88000FC495E80F0084E80F0004F11005A4F571
:107A9800DC740FCC0FC594E80700002386F8603229
:107AA80086F8E232F36986F8A17285E80700C6F81D
:107AB800A23220E085B1A4EB0900C00800041949EE
:107AC80040F00300F9F79AFFD8F800100E484FF479
:107AD8006072BFE7002F9CD1A4EB0900C008000426
:107AE800114940F00200F9F789FF07484FF4607226
:107AF800002101F0D2FC02237360BDE8F08700BFCB
:107B080000F00700F0950700489A002099BE07008A
:107B1800AEBE07004C9A0020A49A00206C9D00205D
:107B280095BF0700D8BE070031BF0700B85900202D
:107B3800C095070070B50C4C054600225821201D41
:107B4800FAF764FA00222060C32104F51870FAF7E6
:107B58005DFA2A46C4F85C022146044B0448BDE895
:107B68007040FFF7CBBE00BF489A0020C89600209F
:107B780000F00700F8B5134B134C144FE41AE4084F
:107B880024040D463A681249064644F00300F9F702
:107B980039FF2846FFF706FF20B90E494FF4C17098
:107BA800FAF750FA32460C4B38682946FFF7A6FE1A
:107BB800024630B144F001000849BDE8F840F9F741
:107BC80021BFF8BDC0950700F0950700B8590020FF
:107BD800C1BF0700EBBF07004893002078C007002B
:107BE8000149FFF7C7BF00BF00F0070038B50546D9
:107BF8000020FFF79FFF044618B903492846FFF7FE
:107C0800B9FF204638BD00BF489A002037B5114B50
:107C1800114C1249E41AE4082404054644F004000F
:107C2800F9F7ECFE2846FFF7BDFA40B10C490246C9
:107C380044F00100F9F7E6FE032003B030BD0190DF
:107C4800FFF7C2FE0198FFF7D1FF0028F5D00549DC
:107C58000246EDE7C0950700F0950700B5C007009C
:107C6800D8C0070003C1070010B5084C4FF40072D4
:107C7800FF2104F15C0001F010FC2022002104F136
:107C8800380001F00AFC0023236310BD489A002045
:107C980029DF704738B50C4D0446D5F8643378B100
:107CA80001330FD1002218210430FAF7AFF9214629
:107CB8002060072205F55970BDE83840FFF7E8BF96
:107CC8000E2038BD0820FCE700F0070050B1064B35
:107CD80003F11C0253F8041B40F8041B9342F9D12A
:107CE800002070470E20704764F3070010B5064C5B
:107CF800002218212046FAF789F954F8043C1B1A87
:107D08005842584110BD00BF68F3070010B50F4C2A
:107D1800D4F82433D4F864231340013313D00C4B24
:107D28000C480D49C01AC008000440F00400F9F7D7
:107D380065FE4FF4FE20FBF7C3FAC92221464FF433
:107D4800FE20FBF7EBFA002010BD00BF489A002088
:107D5800C0950700F89507004EC107002DE9F843C4
:107D6800154B164CDFF86480154E1649E41AE408E2
:107D7800A6EB08062404F60844F004040746324635
:107D88002046F9F73FFE4FF00009B14501D1002523
:107D98000BE058F8393038469847054640B1034655
:107DA80009494A462046F9F736FE2846BDE8F883D1
:107DB80009F10109E9E700BFC0950700C095070070
:107DC800B49507008BC10700AFC10700AC95070049
:107DD8002DE9F843154B164C164D174F1749E41A61
:107DE800E4087F1B2404FF0844F0040406463A46CE
:107DF8002046F9F707FE4FF0000805F10409B845D9
:107E080001D100250BE059F838303046984705462F
:107E180040B103460A4942462046F9F7FCFD284688
:107E2800BDE8F88308F10108E9E700BFC09507003D
:107E3800C0950700AC950700B4950700DBC10700A3
:107E480000C20700034A0023036043608360136392
:107E5800704700BF489A00204FF44053074A5968BA
:107E6800914201BF986800F6FF7020F47F6020F00F
:107E78000F0018BF4FF48050704700BFDBE5B151C9
:107E880008B5FFF7E9FF054B9B69184400F6FF703A
:107E980020F47F6020F00F0008BD00BF489A002042
:107EA8004FF48050704700002DE9F04F89B0064626
:107EB80003920793694A6A4B06919B1ADB081B04D5
:107EC80043F00404674904932046F9F797FD66498F
:107ED800DFF8E081DFF8E091DFF8E0A132462046E4
:107EE800F9F790FD069B6149002B0CBF42464A46B4
:107EF8002046F9F787FD039B5D49002B0CBF4246DE
:107F08004A462046F9F77EFD079B5A49002B0CBFCD
:107F180042464A462046F9F775FD4FF44053564904
:107F28005A68564B20469A4214BF42464A46F9F7C9
:107F380069FD53492046F9F761FDDAF81830DAF897
:107F4800202050492046F9F766FDDAF82430DAF89F
:107F58002C204D492046F9F75EFD4FF0000B5FFAE3
:107F68008BF3BBF1010F02934CD0022B59D0FFF7D2
:107F780087FF039B0546002B42D0DAF82020531ECA
:107F88005A425A410192414FAF4203D24049B1206F
:107F9800FAF758F8069B3F497F1BB74238BF0123C1
:107FA8005A4620460593F9F72DFD3B492A462046B7
:107FB800F9F728FD3949B7422CBF42464A462046C0
:107FC800F9F720FD019B3649002B0CBF42464A4673
:107FD8002046F9F717FD059B3249002B0CBF424696
:107FE8004A462046F9F70EFD059BFBB1019BEBB90C
:107FF8000BF1010BBBF1030FB1D1B74224D217E04B
:10800800039ABFE7FFF728FF079B05463BB94FF4E4
:1080180040521A4B5268D21A18BF0122B2E75A4688
:10802800B0E7012301934FF48055ACE7B74209D27A
:10803800049B1D4943F00200F9F7E0FC042009B055
:10804800BDE8F08F029B33B120461849F9F7D6FCFA
:108058001748FFF7F7FE0020F1E700BFC0950700BB
:10806800C09507002AC2070048C2070068C2070077
:1080780079C2070087C207009CC20700DBE5B1513F
:10808800ACC20700BBC20700DBC2070000E0060065
:10809800FBC2070085C307008FC30700A4C30700FE
:1080A800B9C30700CCC30700DDC3070009C4070034
:1080B800609A002062C207005DC20700489A00204B
:1080C8002DE9F04F4049414E8A6B414DDFF8289128
:1080D800DFF828A1DFF828B185B06F465C31384653
:1080E800FBF7FAFA97E80F004FF0000886E80F0050
:1080F800384BF3604FF447724146284689F80080B0
:10810800CAF80080CBF8008001F0C7F932492A4646
:108118003046FBF77EFD044650B93048304B3149B4
:10812800C01AC008000440F00100F9F767FC14E029
:1081380099F80090B9F1000F04D095F86C312C78BB
:10814800A3B374B1264B25482749C01AC0080004B8
:1081580040F00100F9F752FC0024204605B0BDE8C4
:10816800F08F95F87241002CF7D0DBF80020DAF890
:1081780000103846FBF7B0FA97E80F0086E80F00C2
:108188004FF4B272414605F5BA7001F086F9174905
:1081980005F5BA723046FBF73CFD044680B90F4836
:1081A8000F4B1349C01AC0080004BCE7002CD4D0F8
:1081B800AC79002CD1D008350E4B4C461D60CCE76D
:1081C80005F5BA75F8E700BF489A002014A1002009
:1081D800F89D00209982070078B0070000960700F4
:1081E800C09507001BC4070048C40700C4AF0700B8
:1081F80067C40700D0A10020F49D0020F09D002056
:10820800EC9D002010B590F8553013F0FB0F08D105
:1082180090F864202AB1846E74B30C60012420465F
:1082280010BD13F0010403D090F8564004B1846DDA
:108238009B07F1D590F85C30002BEDD00F4B026E08
:10824800C3F5FC239A4201D81444E5E70C490D48CC
:10825800401AC00800040C4940F00100F9F7DBFBA4
:108268000424074B07480949C01AC008000440F015
:108278000100F9F7C3FBD2E70F24F2E7001007006B
:10828800C095070000960700A3C40700C0C40700F4
:108298005B68DA68134B9A4230B408D1124D2B68E8
:1082A80013B9124C236823B1114B00221A7030BC49
:1082B8007047D0E90131194413F9010B0028A1EBEB
:1082C8000302F9DB2B600A4B0A482260012119706E
:1082D800094B0A49C01AC008000430BC40F0040029
:1082E800F9F790BBC4AF0700F09D0020EC9D00207B
:1082F800F49D002000960700C0950700F1C4070010
:1083080000B591B0FBF7D4FE18B10D49DB20F9F7A1
:1083180099FE0C4920226846FBF71AFF0A490B48C8
:1083280040236A46FBF71CFE18B10549E520F9F71A
:1083380089FE074B01221A7011B05DF804FB00BFDB
:108348000EC5070030A4070024A10020D8A207000A
:10835800C89D00202DE9F047A4B081460E46174677
:10836800984678222023002106A80493DDF8B0A0BF
:1083780001F093F800230593424B1B780BB9FFF7E4
:10838800BFFF4148414C4249241AE408240444F000
:1083980003052846F9F732FB46B944F002003D4987
:1083A800F9F72CFB132024B0BDE8F087B9F1000FD2
:1083B80005D028463849F9F721FB1620F3E7374955
:1083C80052462846F9F71EFB04AB0193344B009341
:1083D80034495346424606A8FBF750FE00284ED1C2
:1083E800402F4CD1304B314606F140021F4651F820
:1083F800040B43F8040B9142F9D12C492846F9F7AC
:10840800FDFA402628482021FBF7AFFE244A049BAA
:108418002749CDE9007605A8FBF7BEFD024640B323
:10842800244944F00100F9F7EDFA44F00400224928
:108438000390F9F7E3FA32461B490398F9F720FB52
:108448001E490398F9F7DAFABDF810201449039881
:10845800F9F716FB1A490398F9F7D0FA194903985E
:108468003246F9F70DFBF9F765F90028FBD105202D
:1084780099E728461449F9F7C1FA012093E70A2039
:1084880091E700BFC89D0020C0950700009607002F
:108498009DC50700C5C50700D9C50700F0C5070079
:1084A8006CA100201CAF07008CA100200BC60700A0
:1084B80024A100201CC607003EC6070049C60700C5
:1084C8004FC6070030A407005BC607004FF44053AF
:1084D8001F4A5B68934213B538D000F500514C68C9
:1084E800A11A4C424C4193422DD100F500525168DB
:1084F800994228D14FF4405316481978142982BF5D
:108508005B691549B3FBF1F3117898BF002314296F
:1085180082BF52691049B2FBF1F21049A0EB010089
:1085280098BF00220E490092C00893424FEA0040CB
:108538000C4A40F0030018BF0A460B4914BF012437
:108548000024F9F772FA204602B010BD0024CAE7E9
:10855800DBE5B1510096070040420F00C0950700C7
:108568006AC6070070C6070076C607002DE9F04303
:10857800ABB006460F4690461C46782220230021C1
:108588000CA8039300F089FF294B1B780BB9FFF760
:10859800B7FE2CB13146202204A8FBF7BDFD04AE7E
:1085A800244B254C2549DFF8AC90E41AE408240450
:1085B80044F0040543463A462846F9F72CFA03AB3B
:1085C80001933A461E49CDF8009043460CA8FBF7A4
:1085D80055FD024640B144F001001A49F9F712FA74
:1085E80000202BB0BDE8F08320223146484600F039
:1085F800F4FED8B1144944F00200F9F7FFF9134921
:108608002846F9F7FBF9202231462846F9F738FAC7
:108618000F492846F9F7F2F9202249462846F9F782
:108628002FFAF9F787F80028FBD1DAE70120D8E715
:10863800C89D0020C095070000960700B6C6070031
:108648001CAF0700E9C607001AC7070034C70700B0
:1086580046C70700C99D002008B5044B986B08B1B0
:10866800FFF72EFD024B187008BD00BF489A002086
:10867800CCA1002010B5044658B1B0F5007F0AD847
:10868800064B00221A70FFF7EFFA054B01209C6396
:1086980010BD0320FCE70420FAE700BFCCA10020AE
:1086A800489A002070B5134C0646E06BA36B42183D
:1086B8009A420D460BD9104B10481149C01AC008F0
:1086C800000440F00100F9F799F9032070BD5C300F
:1086D8000A462044314600F0B7FEE36B04F140023D
:1086E8002B4429463046E363F9F790FC20640120C7
:1086F800ECE700BF489A0020C095070000960700E5
:1087080056C70700014B1878704700BFCCA100205E
:10871800F0B51C4C94F86C2185B07AB394F8D80263
:10872800B4F8DA2204F5377104F5B874164E174D0B
:10873800336800932B68FFF70DFE0128074605D123
:10874800201D00F0CBFA0128074614D01048114C20
:108758001149241AE408240444F00200F9F74EF9F8
:1087680044F004000D490390F9F748F93288296864
:108778000398F9F785F9384605B0F0BD114610465B
:108788000434D3E7F89D0020EC9D0020F09D0020E4
:10879800C09507000096070079C707008FC7070034
:1087A800334BD3E90E329A422DE9F04106460D4685
:1087B8000DD0304B30483149C01AC008000440F091
:1087C8000100F9F71BF908242046BDE8F0812C4F79
:1087D80097F80080B8F1000F09D0FFF751FB294B3B
:1087E800306029461868BDE8F041FFF70BBDFFF778
:1087F80067FC80B3FFF78CFF0128C6F800800446A9
:10880800C5F8008019D11F4B29461868FFF7FAFCF4
:108818000128044611D1034642462868164D4146B0
:10882800FFF742FB134BED1AED082D0440B1164932
:1088380045F00100F9F7E2F80424FFF715FAC3E759
:10884800FFF71EFB11493060024645F00400F9F7B6
:10885800D9F83C70B8E7074B07480D49C01AC0085B
:10886800000440F00100F9F7C9F80524ACE700BF9F
:10887800489A0020C0950700009607009DC707008A
:10888800CCA10020D0A10020B8C70700D3C707009B
:10889800EFC7070037B50D46044630B907490192BE
:1088A8004FF42C70F9F7CEFB019A0123294604F105
:1088B800720003B0BDE83040FFF758BE0EC5070090
:1088C80013B50446084623781146032B2CD8DFE855
:1088D80003F01402161F0022D4F80140F9F796FBA2
:1088E80084420AD01448154B1549C01AC008000420
:1088F800012240F00400F9F785F8012012E00A4649
:1089080000230146601C02B0BDE81040FFF72EBEF0
:10891800034600914022611C0020FFF71BFD431E07
:108928005842584102B010BD40F2D9300549F9F714
:1089380089FB0020F6E700BF00960700C0950700F6
:108948000CC807000EC507002DE9F043A3B0054683
:108958000E461446002178221F4604A820239DF8BD
:10896800AC800393DDF8A89000F097FD4122002128
:10897800284600F092FDB6F89430A34282BF442303
:1089880003FB046393F8968085F80080B8F1030F21
:1089980038D8DFE808F009020F2C0022494638468B
:1089A800F9F734FBC5F801004A4639462846FFF76F
:1089B80087FF19E003AB01936B1C009316494B46E4
:1089C8003A4604A8FBF75AFB0028EDD0FAF7F6FA66
:1089D800124B1349024613481B1ADB081B0443F0C9
:1089E8000100F9F70FF8002023B0BDE8F083442117
:1089F8004C4333199A34B3F898203119681C00F0A5
:108A080023FDD1E70548074B0749C01AC0080004F1
:108A1800424640F00100E4E71CAF0700009607005B
:108A28002FC80700C095070060C807002DE9F04768
:108A3800974B1C68A4B005460F4691460A46014666
:108A48002046FFF727FF002800F0058194F85560BD
:108A5800002E38D14FF0010ACDE9007A2B46324674
:108A6800214613A8FFF770FF002800F00F81B9F125
:108A7800000F46D0DFF82882412213A908F2A1206E
:108A880000F0E2FC834B84488449C8F82CA0C01A43
:108A9800C008000440F00400F8F7B0FF94F89230E2
:108AA800C8F8206013B194F8933013B96368C8F814
:108AB8000830002239462846F9F7A8FA784B0124ED
:108AC800C3E90970C2E04122002102A800F0E5FCD8
:108AD80006F0010A4122002113A806F0020600F060
:108AE800DCFCBAF1000F40F0C080002E40F0A480FA
:108AF8006C4940F26130F9F7A5FAB9F1000F40F07E
:108B08009E80674B01245C61ABE0A36D03F5FF52C7
:108B180003F6FF731F32C3F30B03D31A8A689A4212
:108B280006D25D485B4B6049C01AC0080004A9E042
:108B38004FF440535A68824213D11A78102A88BFDA
:108B48001A690B7898BF0022102B8CBF0B69002381
:108B58009A4206D050484F4B5449C01AC0080004E6
:108B680090E02846FFF7B2FC88B14B4B494A504980
:108B7800A3EB02084FEAD8084FEA084848F0020079
:108B8800F8F73CFF1EB94B4948F001007CE001238F
:108B98000193A36D009300222B46214602A8FFF7FC
:108BA800D3FE002872D0CEB1A26DAB18BA1A00213C
:108BB800CDE9002113A852462146FFF7C5FE00283B
:108BC80064D09DF84C304BB13348324B3A49C01A07
:108BD800C008000440F00200F8F710FFB9F1000FD8
:108BE8008FD0BAF1000F2AD02846FFF76FFC10B1DA
:108BF8003248FFF727F94122314802A900F024FC46
:108C0800274B002E14BFAC22A522DA62A26D5A634C
:108C1800002E3FF44EAF2B48412213A900F014FC5C
:108C280094F8923023B194F89330002B7FF441AF3D
:108C38001B4B6268DA603CE73A462B46B7E7184BAD
:108C4800AA22DA62E4E72048FFF7FCF8FFF70CF8FD
:108C5800134B9D6405E01724B9F1000FF3D1FFF71A
:108C680003F8204624B0BDE8F08705F50051174BFE
:108C7800486898423FF449AF0748064B1449C01A60
:108C8800C008000440F00100F8F7B8FE0524E3E747
:108C9800D0A10020C09507000096070081C80700F2
:108CA800489A00200EC50700FAC8070063C90700E4
:108CB800D0C9070011CA070052CA0700609A0020ED
:108CC800A89C00202A9D00206C9A0020DBE5B15169
:108CD800A9C807000122FFF7A9BE0000F8B504469D
:108CE80018B94D49C420F9F7ADF994F854309BB13F
:108CF80094F8550003280FD894F86E30032B17D03A
:108D0800464B47484749C01AC008000440F00100D4
:108D1800F8F774FE1420F8BD4148404B4249C01A88
:108D2800C008000440F00100F8F768FE0F20F2E7E1
:108D380094F892301BB194F89330002B6AD1237ABF
:108D480033B93748354B3949C01AC0080004E9E738
:108D5800E368342B0BD0314B31483549C01AC00871
:108D6800000440F00200F8F749FE1120D3E74FF461
:108D78004055304A6968238A91422ED143B16269CD
:108D880022B3DBB204F114010022D6B2B3420BD8ED
:108D9800224B23482849C01AC008000440F00200AA
:108DA800F8F72CFE1220B6E751F8047BAE89B742DB
:108DB80002F10102E9D12378B3B90128ABD01848F0
:108DC800164B1E49C01AC0080004ABE710B9012BA6
:108DD800DED1F0E70128EED1DAE713B16369002BA1
:108DE800D6D12378002BD3D001286368144A0ED833
:108DF800926893420ED2094B09481249C01AC0081A
:108E0800000440F00200F8F7F9FD102083E7D2686B
:108E18009342F0D901207EE7A9CA0700C095070050
:108E28000896070053CB07003CCB070066CB07002A
:108E380075CB0700DBE5B15188CB0700ACCB070049
:108E4800489A002098CB070010DF704711DF704761
:108E580013B5044609496846FAF75CF8019808B959
:108E680002B010BDD0E900212046904718B16846ED
:108E7800FAF76AF8F2E71120F2E700BFE4CB07003F
:108E880013B5044607496846FAF744F8019B0BB93D
:108E980002B010BD2046D3E9002190476846FAF792
:108EA80053F8F3E7FCCB0700084B9A6822B11A681D
:108EB80022F480021A607047054B4FF48002C3F811
:108EC8008020BFF34F8FBFF36F8F7047B06B0020C8
:108ED80000E100E00B4991F816335A09EC231341DD
:108EE800DB0706D5084B9A683AB94FF480030B6044
:108EF800704742F20200FBF7A1B91A6842F48002F7
:108F08001A60704700E100E0B06B0020F7B5194F18
:108F18003C7864BB184E012520463570FFF798FF52
:108F2800112821D02046FFF7ABFF144B8DF80340E2
:108F3800186801900DF10300F9F718F8104901A815
:108F4800FFF782FF0446B0FA80F0400938709DF8B8
:108F58000300F9F73BF83CB90A4B34701C70FFF773
:108F6800B9FF2846FFF78CFF204603B0F0BD082460
:108F7800FAE700BFD5A10020D4A10020DFCB07006D
:108F880019420700D6A10020F7B5154F3B781BB34F
:108F9800144E01203070FFF75BFF11284FF00005D9
:108FA8001CD00220FFF76CFF0DF107008DF8075069
:108FB800F8F7DCFFFFF74AFF04469DF807003D700D
:108FC800F9F704F82CB903203470FFF76DFFFFF7A9
:108FD80057FF204603B0F0BD0824FAE72C46F8E70F
:108FE800D5A10020D4A10020054B1B7833B1054B37
:108FF8001B780BB1FFF7C8BFFFF788BF0820704781
:10900800D4A10020D5A10020014B1878704700BFDB
:10901800D5A1002007B508496846F9F77BFF019BF1
:1090280013B903B05DF804FBD3E900209047684604
:10903800F9F78AFFF3E700BFF0CB0700FFF7EABFB5
:1090480060DF704769DF704761DF704730B5134DE7
:10905800ADF5017D4FF4FA740DF1020103A8ADF8E6
:109068000240FFF7F1FF70B9294601A8F9F752FF4E
:10907800029B002BF0D003A8D3E90021904701A858
:10908800F9F762FFF4E7052805D00DF5017DBDE885
:109098003040FBF7D3B80DF5017D30BD84CE070015
:1090A800024B1B780BB1FFF7D1BF7047D7A1002047
:1090B80018B1034B0360002070470E20704700BFB3
:1090C8006859002030B5054685B00C46002900F0E7
:1090D800A4800023CDE90133514A039301230A6098
:1090E8008DF804008DF8063001A906232020ADF87C
:1090F8000830FFF7A7FF60B1F9F760FF494B4A490D
:1091080002464A481B1ADB081B0443F00100F8F723
:1091180079FC0023CDE9013303932268012301A9D7
:1091280040208DF80530FFF78DFF60B1F9F746FF55
:109138003C4B3F4902463D481B1ADB081B0443F0E1
:109148000100F8F75FFC0023CDE90133039322689F
:109158008DF80450F72301A92320ADF80630FFF756
:1091680071FF60B1F9F72AFF2E4B324902462F48AA
:109178001B1ADB081B0443F00100F8F743FC00232B
:1091880001202268039301A9CDE901338DF8040079
:10919800FFF758FF60B1F9F711FF224B2649024645
:1091A80022481B1ADB081B0443F00100F8F72AFCCD
:1091B8000023CDE9023322684FF4B06301A9A1204E
:1091C8000193FFF73FFF60B1F9F7F8FE154B1B4914
:1091D800024616481B1ADB081B0443F00100F8F787
:1091E80011FC00252268039501A9A020CDE90155AD
:1091F800FFF728FF034668B1F9F7E0FE094B10496D
:1092080002460A481B1ADB081B0443F00100F8F762
:10921800F9FB2B46184605B030BD0E23FAE700BF10
:10922800685900202096070008CC0700C095070061
:109238004ECC07009ACC0700E1CC07002DCD0700E3
:109248007ECD070073B505460668FFF7F9FE2B6863
:10925800B34204461DD91A481A4B1B491B1ADB088E
:109268001B0443F002000190F8F7C8FB2B6817496C
:1092780001983246F8F7CFFB4FF080532A68D3F8AD
:109288000C31134901989B0203F100539A1AF8F71D
:10929800B9FB2CB90F4B01221A70204602B070BDE1
:1092A8002046F9F78BFE074B0B49024604481B1A68
:1092B800DB081B0443F00100F8F7A4FBEDE700BF4F
:1092C800C095070020960700D1CD070000CE070003
:1092D80031CE0700D7A100205BCE07004BDF7047D7
:1092E8001FB50E4C01A8FFF7F9FF70B9214602A877
:1092F800F9F710FE039B002BF4D00198D3E9002165
:10930800904702A8F9F720FEF4E7052804D004B036
:10931800BDE81040FAF792BF04B010BD9CCE07001C
:109328007F2805D8034B185C034B5B5C18407047DB
:1093380000207047B4CE070034CF0700A0F16103C6
:10934800192B98BF20387047A0F14103192B98BFFB
:10935800203070477F2805D8034B185C034B5B5CB3
:109368001840704700207047B4CE070034CF07007C
:10937800A0F16103192B98BF20387047A0F1410371
:10938800192B98BF203070477F299ABF01700120A0
:109398006FF02E0070475AB10A787F2A0AD800B1B8
:1093A8000260002119605960501A18BF01207047E7
:1093B800002070476FF02E007047000008B5034B7F
:1093C8005B689B681B68984708BD00BFBC590020B4
:1093D80008B50921FFF7F2FF08BD9AB330B59446E6
:1093E8000F2A18D902460B4640EA010414F0030F6D
:1093F80002D00CF1FF3C11E0194610460432043348
:109408000C680568A54206D110461946ACF1040C53
:10941800BCF1040FF0D8BCF1010C0FD00A4603468A
:1094280084441146184601330132047891F800E06B
:10943800744503D1184611466345F2D100780B787C
:10944800C01A30BD00207047844640EA010313F07B
:10945800030F18D18446202A0BD32DE9F007B1E871
:10946800F807A0E8F807A2F12002202AF7D2BDE801
:10947800F007042A07D351F8043B40F8043BA2F153
:109488000402042AF7D2002A05D011F8013B00F89B
:10949800013B013AF9D1604670478446002A2DD035
:1094A80010F0030F04D000F8011B013A26D0F7E7AB
:1094B800C9B241EA012141EA0141202A12D3A2F1AD
:1094C80020022DE9F0030B460C460D460E460F46CA
:1094D80088468946A0E8FA03203AFBD2BDE8F003A3
:1094E80020320BD0042A05D340F8041B043A05D0D7
:1094F800042AF9D200F8011B013AFBD160467047F3
:10950800024610F0030F16D111F0030F13D12DE905
:10951800F0004FF001374FF0803351F8044BA4EBC3
:10952800070525EA04051D4002D142F8044BF4E77B
:10953800A1F10401F0BC11F8013B02F8013B002B3A
:10954800F9D1704700F1010110F0030F11D010F8A4
:10955800012B002A23D010F0030F0AD010F8012B9A
:10956800002A1CD010F0030F03D010F8012B002A9A
:1095780015D02DE970004FF001324FF0803350F8CC
:10958800044BA4EB020525EA04051D4000D1F6E7CB
:10959800A0F1040070BC10F8012B002AFBD1A0EB4D
:0495A8000100704707
:0895AC00916F0700516C0700EC
:0C95B40000000000030000003D3E070026
:1095C000F997070000000404589907000000000004
:1095D000FDAE07000000040489B607000000040483
:1095E00054B8070000000404BDBD070000000404D7
:1095F0003DC107000000040475C107000000040419
:1096000096CA070000000404C0CB07000000040451
:10961000649B070000000404D7CB0700000003038D
:1096200078CE07000000030390CE0700000003037C
:10963000145A0020DC5A0020E45A00201C5A002052
:1096400018000000A4820020E0920020F192002087
:08965000AC820020F4000000D0
:10965800B896070000000000529707007C590020C8
:08966800B966070000000000D4
:08967000C12A07000000000000
:08967800812C07000000000036
:10968000A990070000000000E99207000000000018
:08969000752C0700000000002A
:109698000000000000000000257107000010000015
:0496A80000000800B6
:1096AC00000000000338FDD870470000BD13070010
:1096BC0029140700B9130700443A5C576F726B5FAB
:1096CC004A616B756A615C5355484F5F494D414720
:1096DC00455C31315F454D455247454E43595F53CB
:1096EC0057495443485C23544F4F4C535C7372633B
:1096FC005F32303231313231395C30315F64667512
:10970C005F626C652E32303231313231395C636FCD
:10971C006D706F6E656E74735C6C69627261726988
:10972C0065735C6C6F675C7372635C6E72665F6CA6
:10973C006F675F64656661756C745F6261636B65AE
:10974C006E64732E63007274745F6C6F675F62611A
:10975C00636B656E6400443A5C576F726B5F4A6171
:10976C006B756A615C5355484F5F494D4147455C89
:10977C0031315F454D455247454E43595F5357492B
:10978C005443485C23544F4F4C535C7372635F32A9
:10979C00303231313231395C30315F6466755F6241
:1097AC006C652E32303231313231395C636F6D7011
:1097BC006F6E656E74735C6C6962726172696573ED
:1097CC005C6C6F675C7372635C6E72665F6C6F6708
:1097DC005F66726F6E74656E642E63004261636BBC
:1097EC00656E647320666C75736865640061707077
:1097FC0000000000046B00207F000000846B002040
:10980C001B5B313B33316D0025734C6F67732064E8
:10981C00726F70706564202825642925730D0A0009
:10982C001B5B306D003C25733E2025733A200020D5
:10983C002530327800202020007C002563001B5B43
:10984C00313B33306D001B5B313B33326D001B5BA6
:10985C00313B33336D001B5B313B33346D001B5B91
:10986C00313B33356D001B5B313B33366D001B5B7D
:10987C00313B33376D006572726F72007761726EB7
:10988C00696E6700696E666F0064656275670000DB
:10989C002C9807004A9807000C980700529807006C
:1098AC005A980700629807006A9807007298070098
:1098BC007A9807000000000082980700889807003B
:1098CC009098070095980700443A5C576F726B5F4D
:1098DC004A616B756A615C5355484F5F494D41470E
:1098EC00455C31315F454D455247454E43595F53B9
:1098FC0057495443485C23544F4F4C535C73726329
:10990C005F32303231313231395C30315F646675FF
:10991C005F626C652E32303231313231395C636FBB
:10992C006D706F6E656E74735C6C69627261726976
:10993C0065735C7574696C5C6170705F7574696C6F
:10994C005F706C6174666F726D2E63006D656D5F18
:10995C006D6E677200443A5C576F726B5F4A616B55
:10996C00756A615C5355484F5F494D4147455C31C1
:10997C00315F454D455247454E43595F5357495406
:10998C0043485C23544F4F4C535C7372635F3230CB
:10999C003231313231395C30315F6466755F626C03
:1099AC00652E32303231313231395C636F6D706F0C
:1099BC006E656E74735C6C69627261726965735CFE
:1099CC0062616C6C6F635C6E72665F62616C6C6F13
:1099DC00632E6300443A5C576F726B5F4A616B7520
:1099EC006A615C5355484F5F494D4147455C313185
:1099FC005F454D455247454E43595F535749544374
:109A0C00485C23544F4F4C535C7372635F3230325B
:109A1C0031313231395C30315F6466755F626C654F
:109A2C002E32303231313231395C65787465726E78
:109A3C00616C5C667072696E74665C6E72665F6691
:109A4C007072696E74662E6300443A5C576F726B69
:109A5C005F4A616B756A615C5355484F5F494D4174
:109A6C0047455C31315F454D455247454E43595F43
:109A7C005357495443485C23544F4F4C535C7372B7
:109A8C00635F32303231313231395C30315F646690
:109A9C00755F626C652E32303231313231395C6532
:109AAC00787465726E616C5C667072696E74665CFB
:109ABC006E72665F667072696E74665F666F726DE9
:109ACC0061742E63003031323334353637383941D6
:109ADC004243444546443A5C576F726B5F4A616B34
:109AEC00756A615C5355484F5F494D4147455C3140
:109AFC00315F454D455247454E43595F5357495485
:109B0C0043485C23544F4F4C535C7372635F323049
:109B1C003231313231395C30315F6466755F626C81
:109B2C00652E32303231313231395C636F6D706F8A
:109B3C006E656E74735C6C69627261726965735C7C
:109B4C006673746F726167655C6E72665F66737460
:109B5C006F726167652E63006E72665F6673746FF9
:109B6C007261676500000000001000000400000036
:109B7C0001000000592907007D2907008D290700E5
:109B8C009D290700F12907006529070069290700AD
:109B9C006D29070000100000040000000100000007
:109BAC00052B0700E52A0700D52A0700112D070011
:109BBC00C12C0700A92A0700AD2A0700B12A07000B
:109BCC00443A5C576F726B5F4A616B756A615C53A8
:109BDC0055484F5F494D4147455C31315F454D45D7
:109BEC005247454E43595F5357495443485C23549D
:109BFC004F4F4C535C7372635F32303231313231C0
:109C0C00395C30315F6466755F626C652E32303260
:109C1C0031313231395C636F6D706F6E656E747398
:109C2C005C6C69627261726965735C6D656D6F62A3
:109C3C006A5C6E72665F6D656D6F626A2E6300445E
:109C4C003A5C576F726B5F4A616B756A615C535516
:109C5C00484F5F494D4147455C31315F454D455259
:109C6C0047454E43595F5357495443485C23544F1F
:109C7C004F4C535C7372635F323032313132313955
:109C8C005C30315F6466755F626C652E32303231E8
:109C9C00313231395C636F6D706F6E656E74735CED
:109CAC006C69627261726965735C65787065726902
:109CBC006D656E74616C5F73656374696F6E5F76EE
:109CCC006172735C6E72665F73656374696F6E5FED
:109CDC00697465722E63004E52465F53554343457B
:109CEC005353004E52465F4552524F525F535643A8
:109CFC005F48414E444C45525F4D495353494E4782
:109D0C00004E52465F4552524F525F534F46544499
:109D1C0045564943455F4E4F545F454E41424C4575
:109D2C0044004E52465F4552524F525F494E544585
:109D3C00524E414C004E52465F4552524F525F4E6E
:109D4C004F5F4D454D004E52465F4552524F525F4C
:109D5C004E4F545F464F554E44004E52465F45524F
:109D6C00524F525F4E4F545F535550504F525445C3
:109D7C0044004E52465F4552524F525F494E564137
:109D8C004C49445F504152414D004E52465F455242
:109D9C00524F525F494E56414C49445F53544154C3
:109DAC0045004E52465F4552524F525F494E564106
:109DBC004C49445F4C454E475448004E52465F4513
:109DCC0052524F525F494E56414C49445F464C41AA
:109DDC004753004E52465F4552524F525F494E56C2
:109DEC00414C49445F44415441004E52465F4552F8
:109DFC00524F525F444154415F53495A45004E52B1
:109E0C00465F4552524F525F54494D454F55540091
:109E1C004E52465F4552524F525F4E554C4C004E7F
:109E2C0052465F4552524F525F464F52424944444C
:109E3C00454E004E52465F4552524F525F494E5668
:109E4C00414C49445F41444452004E52465F455296
:109E5C00524F525F42555359004E52465F45525233
:109E6C004F525F434F4E4E5F434F554E54004E5230
:109E7C00465F4552524F525F5245534F55524345E0
:109E8C0053004E52465F4552524F525F4D4F445510
:109E9C004C455F4E4F545F494E495449414C495AC9
:109EAC004544004E52465F4552524F525F4D5554F9
:109EBC0045585F494E49545F4641494C4544004E14
:109ECC0052465F4552524F525F4D555445585F4C68
:109EDC004F434B5F4641494C4544004E52465F450B
:109EEC0052524F525F4D555445585F554E4C4F434F
:109EFC004B5F4641494C4544004E52465F455252D9
:109F0C004F525F4D555445585F434F4E445F494E39
:109F1C0049545F4641494C4544004E52465F4552B8
:109F2C00524F525F4D4F44554C455F414C52454149
:109F3C0044595F494E495449414C495A4544004E95
:109F4C0052465F4552524F525F53544F5241474510
:109F5C005F46554C4C004E52465F4552524F525F35
:109F6C004150495F4E4F545F494D504C454D454E05
:109F7C00544544004E52465F4552524F525F46453F
:109F8C0041545552455F4E4F545F454E41424C45EE
:109F9C0044004E52465F4552524F525F494F5F50FC
:109FAC00454E44494E47004E52465F4552524F5221
:109FBC005F4452565F5457495F4552525F4F564566
:109FCC005252554E004E52465F4552524F525F44CC
:109FDC0052565F5457495F4552525F414E41434B75
:109FEC00004E52465F4552524F525F4452565F5498
:109FFC0057495F4552525F444E41434B004E5246C7
:10A00C005F4552524F525F424C455F495053505F2F
:10A01C0052585F504B545F5452554E434154454433
:10A02C00004E52465F4552524F525F424C455F497B
:10A03C005053505F4348414E4E454C5F414C524546
:10A04C004144595F455849535453004E52465F455D
:10A05C0052524F525F424C455F495053505F4C49EE
:10A06C004E4B5F444953434F4E4E45435445440079
:10A07C004E52465F4552524F525F424C455F4950DB
:10A08C0053505F504545525F52454A4543544544F1
:10A09C0000556E6B6E6F776E206572726F722063F7
:10A0AC006F64650000000000E39C070001000000E5
:10A0BC00EF9C0700020000000D9D0700030000004C
:10A0CC002E9D070004000000419D070005000000C4
:10A0DC00529D070006000000669D07000700000067
:10A0EC007E9D070008000000969D070009000000F7
:10A0FC00AE9D07000A000000C79D07000B00000082
:10A10C00DF9D07000C000000F69D07000D0000000D
:10A11C000A9E07000E0000001C9E07000F000000A6
:10A12C002B9E0700100000003F9E0700110000004E
:10A13C00569E070012000000659E070013000000E9
:10A14C007A9E0700800000008E9E070081000000B0
:10A15C00AF9E070082000000CB9E0700830000002A
:10A16C00E79E070084000000059F070085000000A3
:10A17C00269F0700860000004B9F07009000000000
:10A18C00629F070091000000809F07009200000072
:10A19C009E9F070000820000B39F07000182000011
:10A1AC00D19F070002820000ED9F07000084000091
:10A1BC0009A00700018400002DA007000284000004
:10A1CC0057A00700038400007CA00700982F8A4248
:10A1DC0091443771CFFBC0B5A5DBB5E95BC25639ED
:10A1EC00F111F159A4823F92D55E1CAB98AA07D805
:10A1FC00015B8312BE853124C37D0C55745DBE7228
:10A20C00FEB1DE80A706DC9B74F19BC1C1699BE4A7
:10A21C008647BEEFC69DC10FCCA10C246F2CE92D37
:10A22C00AA84744ADCA9B05CDA88F97652513E985B
:10A23C006DC631A8C82703B0C77F59BFF30BE0C662
:10A24C004791A7D55163CA0667292914850AB727F0
:10A25C0038211B2EFC6D2C4D130D385354730A658D
:10A26C00BB0A6A762EC9C281852C7292A1E8BFA264
:10A27C004B661AA8708B4BC2A3516CC719E892D1CC
:10A28C00240699D685350EF470A06A1016C1A4194F
:10A29C00086C371E4C774827B5BCB034B30C1C394E
:10A2AC004AAAD84E4FCA9C5BF36F2E68EE828F740D
:10A2BC006F63A5781478C8840802C78CFAFFBE9027
:10A2CC00EB6C50A4F7A3F9BEF27871C648002800D5
:10A2DC0000204000C54F0700A93707004F37070083
:10A2EC009F3C07000F3D07002F3D07009F360700DE
:10A2FC00613607003B3C0700000000002E2E2F2E7D
:10A30C002E2F2E2E2F2E2E2F2E2E2F6D6F64756C22
:10A31C0065732F6E7266782F68616C2F6E72665F34
:10A32C006770696F2E6800443A5C576F726B5F4AB6
:10A33C00616B756A615C5355484F5F494D414745A8
:10A34C005C31315F454D455247454E43595F53573C
:10A35C00495443485C23544F4F4C535C7372635FB6
:10A36C0032303231313231395C30315F6466755F95
:10A37C00626C652E32303231313231395C636F6D43
:10A38C00706F6E656E74735C626F617264735C6225
:10A39C006F617264732E630011121314443A5C578C
:10A3AC006F726B5F4A616B756A615C5355484F5FA6
:10A3BC00494D4147455C31315F454D455247454E0E
:10A3CC0043595F5357495443485C23544F4F4C53A4
:10A3DC005C7372635F32303231313231395C30311F
:10A3EC005F6466755F626C652E32303231313231AA
:10A3FC00395C636F6D706F6E656E74735C6C6962E3
:10A40C007261726965735C63727970746F5C6E7281
:10A41C00665F63727970746F5F7368617265642EC6
:10A42C00630000001D85DB303598B491A49E842B0D
:10A43C008A8FAC713F6865700F349CBD1C79B71066
:10A44C0000F1C9B563F941D170D673CEDCF7EC4895
:10A45C007D99B0EF9297D28B1DD0FFDE6A7C7ABFCC
:10A46C00604DD71F5265636569766564206120660F
:10A47C0061756C74212069643A2030782530387805
:10A48C002C2070633A203078253038782C20696E77
:10A49C00666F3A20307825303878005265636569EC
:10A4AC0076656420616E206572726F723A20307826
:10A4BC00253038782100496E73696465206D6169B7
:10A4CC006E004166746572206D61696E2C20736834
:10A4DC006F756C64206E657665722062652072659E
:10A4EC0061636865642E000000000000000000003D
:10A4FC00000000000338FDD8704700000820000160
:10A50C00FFFFFFFFFFFFFFFFFFFFFFFF000000004B
:10A51C00000000000000000001000000FFFFFFFF32
:10A52C00512563FCC2CAB9F3849E17A7ADFAE6BCE9
:10A53C00FFFFFFFFFFFFFFFF00000000FFFFFFFF1B
:10A54C0096C298D84539A1F4A033EB2D817D0377C1
:10A55C00F240A463E5E6BCF847422CE1F2D1176B5C
:10A56C00F551BF376840B6CBCE5E316B5733CE2B2F
:10A57C00169E0F7C4AEBE78E9B7F1AFEE242E34F5E
:10A58C004B60D2273E3CCE3BF6B053CCB0061D659B
:10A59C00BC86987655BDEBB3E7933AAAD835C65A24
:10A5AC008B490700DD4A07003D4B07005465726D6F
:10A5BC00696E616C00525454005345474745520034
:10A5CC00526573657474696E6720626F6F746C6F1B
:10A5DC00616465722E00496E616374697669747981
:10A5EC002074696D656F75742E00696E20776561D6
:10A5FC006B206E72665F6466755F696E69745F75F9
:10A60C0073657200476574206264206164647265CE
:10A61C00737320746F3A202530325820253032580D
:10A62C00202530325800496E206E72665F626F6F63
:10A63C00746C6F616465725F696E697400426F6FF0
:10A64C00742076616C69646174696F6E20666169EF
:10A65C006C65642E204E6F2076616C69642061708D
:10A66C007020746F20626F6F742E00426F6F7420B5
:10A67C0076616C69646174696F6E206661696C6582
:10A68C00642E20536F667444657669636520697324
:10A69C002070726573656E742062757420696E76B5
:10A6AC00616C69642E00426F6F742076616C696412
:10A6BC006174696F6E206661696C65642E204170EF
:10A6CC007020697320696E76616C69642E0041702C
:10A6DC00702069732076616C696400444655206D66
:10A6EC006F646520626563617573652061707020AD
:10A6FC006973206E6F742076616C69642E00444619
:10A70C0055206D6F64652072657175657374656431
:10A71C002076696120627574746F6E2E0044465504
:10A72C00206D6F6465207265717565737465642046
:10A73C007669612047505245475245542E00556E5C
:10A74C00726561636861626C65003D3D3D3D3D3DF8
:10A75C003D3D3D3D3D3D3D00456E746572206D6156
:10A76C00696E206C6F6F7000443A5C576F726B5F50
:10A77C004A616B756A615C5355484F5F494D41475F
:10A78C00455C31315F454D455247454E43595F530A
:10A79C0057495443485C23544F4F4C535C7372637A
:10A7AC005F32303231313231395C30315F64667551
:10A7BC005F626C652E32303231313231395C636F0D
:10A7CC006D706F6E656E74735C6C696272617269C8
:10A7DC0065735C626F6F746C6F616465725C6E72D2
:10A7EC00665F626F6F746C6F616465722E6300528A
:10A7FC00756E6E696E67206E72665F626F6F746CD9
:10A80C006F616465725F6170705F737461727420E4
:10A81C007769746820616464726573733A20307868
:10A82C00253038780044697361626C696E67206901
:10A83C006E74657272757074732E204E5649432D6A
:10A84C003E494345525B305D3A20307825780046CE
:10A85C0061696C65642072756E6E696E67206E72CC
:10A86C00665F6466755F6D62725F6972715F666F59
:10A87C0072776172645F616464726573735F736530
:10A88C0074282900436F756C64206E6F742070728D
:10A89C006F7465637420626F6F746C6F6164657242
:10A8AC0020616E642073657474696E6773207061C7
:10A8BC006765732C20307825782E00436F756C6497
:10A8CC00206E6F742070726F7465637420536F66A2
:10A8DC007444657669636520616E64206170706C88
:10A8EC0069636174696F6E2C20307825782E004472
:10A8FC003A5C576F726B5F4A616B756A615C53555A
:10A90C00484F5F494D4147455C31315F454D45529C
:10A91C0047454E43595F5357495443485C23544F62
:10A92C004F4C535C7372635F323032313132313998
:10A93C005C30315F6466755F626C652E323032312B
:10A94C00313231395C636F6D706F6E656E74735C30
:10A95C006C69627261726965735C626F6F746C6F43
:10A96C00616465725C6E72665F626F6F746C6F614E
:10A97C006465725F6170705F73746172745F666935
:10A98C006E616C2E630074696D65725F61637469CE
:10A99C00766174652028307825782900443A5C5714
:10A9AC006F726B5F4A616B756A615C5355484F5FA0
:10A9BC00494D4147455C31315F454D455247454E08
:10A9CC0043595F5357495443485C23544F4F4C539E
:10A9DC005C7372635F32303231313231395C303119
:10A9EC005F6466755F626C652E32303231313231A4
:10A9FC00395C636F6D706F6E656E74735C6C6962DD
:10AA0C007261726965735C626F6F746C6F6164659F
:10AA1C00725C6E72665F626F6F746C6F616465728C
:10AA2C005F6466755F74696D6572732E630074691B
:10AA3C006D65725F73746F702028307825782900EB
:10AA4C0074696D65725F6669726520283078257847
:10AA5C00290000000338FDD8704756657269667985
:10AA6C00696E6720424C3A20416464723A20307817
:10AA7C00253038782C205372633A203078253038C2
:10AA8C00782C204C656E3A2030782530387800438D
:10AA9C006F7079696E6720626F6F746C6F6164653B
:10AAAC00723A205372633A203078253038782C2053
:10AABC004C656E3A20307825303878004E6F206225
:10AACC006F6F746C6F6164657220636F7079206E48
:10AADC0065656465642C20626F6F746C6F6164656E
:10AAEC00722075706461746520636F6D706C657431
:10AAFC00652E005265717565737420746F20636FD9
:10AB0C00707920424C206661696C6564004E6F2040
:10AB1C00636F7079206E656564656400443A5C57B8
:10AB2C006F726B5F4A616B756A615C5355484F5F1E
:10AB3C00494D4147455C31315F454D455247454E86
:10AB4C0043595F5357495443485C23544F4F4C531C
:10AB5C005C7372635F32303231313231395C303197
:10AB6C005F6466755F626C652E3230323131323122
:10AB7C00395C636F6D706F6E656E74735C6C69625B
:10AB8C007261726965735C626F6F746C6F6164651E
:10AB9C00725C6E72665F626F6F746C6F616465720B
:10ABAC005F66775F61637469766174696F6E2E633B
:10ABBC0000436F7079696E67203078257820746F48
:10ABCC0020307825782C2073697A653A20307825E6
:10ABDC0078004661696C656420746F2077726974C3
:10ABEC006520696D61676520636F7079696E672098
:10ABFC0070726F677265737320746F2073657474F1
:10AC0C00696E677320706167652E00456E7465729E
:10AC1C00206E72665F626F6F746C6F616465725FD9
:10AC2C006466755F73645F636F6E74696E756500DF
:10AC3C00536F75726365206164647265737320640D
:10AC4C006F6573206E6F7420636F6E7461696E2014
:10AC5C00612076616C696420536F66744465766913
:10AC6C0063652E00534420616C72656164792063C6
:10AC7C006F70696564005570646174696E67205308
:10AC8C00442E204F6C64205344207665723A202564
:10AC9C00642C204E6577207665723A202564004638
:10ACAC0061696C656420746F20636F7079206669CC
:10ACBC00726D776172652E00456E746572206E72CE
:10ACCC00665F626F6F746C6F616465725F66775FED
:10ACDC0061637469766174650056616C69642041C6
:10ACEC00707000456E746572206E72665F64667576
:10ACFC005F6170705F636F6E74696E75650053652C
:10AD0C007474696E67206170702061732076616C59
:10AD1C0069640043524320636F6D7075746174698C
:10AD2C006F6E206661696C656420666F7220636F5C
:10AD3C0070696564206170703A207372632063726D
:10AD4C00633A203078253038782C20726573206374
:10AD5C0072633A203078253038780056616C69641B
:10AD6C002053440056616C696420424C0056616C5F
:10AD7C006964205344202B20424C00456E7465724C
:10AD8C00206E72665F6466755F73645F626C5F638E
:10AD9C006F6E74696E75650053442B424C3A2053A8
:10ADAC004420636F7079206661696C65640053445C
:10ADBC002B424C3A20424C20636F707920666169BB
:10ADCC006C6564004E6F206669726D7761726520E8
:10ADDC00746F2061637469766174652E00416374CD
:10ADEC0069766174696F6E206661696C6564207741
:10ADFC00697468206572726F722025642028626104
:10AE0C006E6B20636F64653A203078257829004199
:10AE1C0020536F667444657669636520686173209E
:10AE2C006A757374206265656E20616374697661FE
:10AE3C007465642E2049742773206C696B656C797A
:10AE4C00207468617420616E206170706C6963613C
:10AE5C0074696F6E2077696C6C20636F6D65206907
:10AE6C006D6D6564696174656C7900436F756C64B4
:10AE7C00206E6F74207772697465207365747469C1
:10AE8C006E67732E00496E7465726E616C20666518
:10AE9C0065640057445420656E61626C65642043A0
:10AEAC0052563A2564207469636B73005374617253
:10AEBC0074696E6720612074696D65722028256441
:10AECC00207469636B732920666F722066656564F4
:10AEDC00696E67207761746368646F672E005744EE
:10AEEC0054206973206E6F7420656E61626C6564AA
:10AEFC00006E72665F626F6F746C6F616465725F17
:10AF0C0077647400000001010000000101000000E2
:10AF1C00DB640700D5640700B5640700200000005F
:10AF2C00780000000000000001000100000000009B
:10AF3C0001000000000000000200050001000000FC
:10AF4C0042000000000000000000000000000000B3
:10AF5C000000000000000000010011000100FFFFD4
:10AF6C000100000000000000020017000200FEFFBC
:10AF7C0064010000C4AF07000000000000000000E6
:10AF8C0000000000000000000100010000000000B3
:10AF9C00010000000000000002000500010000009C
:10AFAC002200000000000000000000000000000073
:10AFBC000000000000000000010011000400FCFF74
:10AFCC000400000000000000020011000400FCFF5F
:10AFDC000400000000000000030021000400FCFF3E
:10AFEC000400100000000000040011000100FFFF2D
:10AFFC000100000000000000050011000200FEFF2F
:10B00C000400000000000000060011000400FCFF1A
:10B01C000400000000000000070011000400FCFF09
:10B02C000400000000000000080017000200FEFFF2
:10B03C002400000094AF0700090010000100FFFF7E
:10B04C000100000074B007000A0027000200FEFF98
:10B05C004400030034AF07000000000000000000B3
:10B06C0000000000000000000000000001001700BC
:10B07C000400FCFF6801000064AF07000200170029
:10B08C000400FCFFAC010000A8B0070000000000A9
:10B09C00000000000000000000000000010007009C
:10B0AC00000000006801000064AF0700020001000E
:10B0BC00000000000100000000000000030005007B
:10B0CC000100000042000000000000000000000031
:10B0DC00000000000000000000000000456E7465D8
:10B0EC0072696E6720444655206D6F64652E00436F
:10B0FC006F756C64206E6F7420696E6974616C6915
:10B10C007A6520444655207472616E73706F727448
:10B11C003A203078253038780046726565696E675C
:10B12C0020627566666572202570004164766572D2
:10B13C00746973696E672E2E2E00436F6E6E656395
:10B14C00746564004661696C75726520746F207556
:10B15C00706461746520636F6E6E656374696F6E85
:10B16C0020706172616D65746572733A2030782558
:10B17C00780063616E6E6F7420616C6C6F636174C8
:10B18C0065206D656D6F72792062756666657221DA
:10B19C000042756666657220257020616371756961
:10B1AC007265642C206C656E20256420282564292A
:10B1BC0000526563656976656420424C455F474182
:10B1CC005454535F4556545F45584348414E474588
:10B1DC005F4D54555F524551554553542028726567
:10B1EC0071756573743A2025642C207265706C79C6
:10B1FC003A202564292E00526563656976656420C2
:10B20C00424C455F4741505F4556545F4441544161
:10B21C005F4C454E4754485F5550444154455F522E
:10B22C004551554553542E005265636569766564E6
:10B23C0020424C455F4741505F4556545F44415452
:10B24C00415F4C454E4754485F555044415445204E
:10B25C002825752C206D61785F72785F74696D6537
:10B26C00202575292E005265636569766564204238
:10B27C004C455F4741505F4556545F5345435F50C3
:10B28C004152414D535F5245515545535400434330
:10B29C00434420666F722073657276696365206320
:10B2AC0068616E6765642069732030782530347866
:10B2BC0000526563656976656420424C455F474181
:10B2CC00505F4556545F434F4E4E5F504152414D77
:10B2DC005F555044415445006D61785F636F6E6EED
:10B2EC005F696E74657276616C3A202564006D69D5
:10B2FC006E5F636F6E6E5F696E74657276616C3AC9
:10B30C0020256400736C6176655F6C6174656E6397
:10B31C00793A20256400636F6E6E5F7375705F748D
:10B32C00696D656F75743A202564005265636569B3
:10B33C0076656420424C455F4741505F4556545FEB
:10B34C00434F4E4E5F504152414D5F555044415416
:10B35C00455F52455155455354004661696C7572B1
:10B36C006520746F2075706461746520636F6E6EF8
:10B37C00656374696F6E20706172616D657465725E
:10B38C0020726571756573743A2030782578005297
:10B39C006563656976656420424C455F4741505F43
:10B3AC004556545F5048595F5550444154452028E8
:10B3BC0052583A25642C2054583A25642C20737426
:10B3CC00617475733A256429005265636569766505
:10B3DC006420424C455F4741505F4556545F50488E
:10B3EC00595F5550444154455F524551554553544E
:10B3FC002E005365742072656365697074206E6FDE
:10B40C0074696600436F756C64206E6F742068619C
:10B41C006E646C65206F6E5F6374726C5F70745FCA
:10B42C0077726974652E206572725F636F64653A1A
:10B43C002030782530347800526563656976656410
:10B44C0020424C455F4741505F4556545F5345433E
:10B45C005F494E464F5F524551554553540046691E
:10B46C006E69736865642068616E646C696E6720D0
:10B47C00636F6E6E20736563207570646174650014
:10B48C005368757474696E6720646F776E20424CD4
:10B49C0045207472616E73706F72742E0044697300
:10B4AC00636F6E6E656374696E672E00424C452047
:10B4BC007472616E73706F7274207368757420642B
:10B4CC006F776E2E00443A5C576F726B5F4A616BFC
:10B4DC00756A615C5355484F5F494D4147455C3136
:10B4EC00315F454D455247454E43595F535749547B
:10B4FC0043485C23544F4F4C535C7372635F323040
:10B50C003231313231395C30315F6466755F626C77
:10B51C00652E32303231313231395C636F6D706F80
:10B52C006E656E74735C6C69627261726965735C72
:10B53C00626F6F746C6F616465725C626C655F6482
:10B54C0066755C6E72665F6466755F626C652E63B1
:10B55C00004446552072657175657374202564200E
:10B56C006661696C65642077697468206572726FB6
:10B57C00723A2030782578004945532D32303042CC
:10B58C0000496E697469616C697A696E6720424C16
:10B59C004520444655207472616E73706F7274004E
:10B5AC0053657474696E6720757020766563746F6B
:10B5BC0072207461626C653A2030782530387800DE
:10B5CC00456E61626C696E6720536F667444657674
:10B5DC006963652E00436F6E6669677572696E6785
:10B5EC0020424C4520737461636B2E00456E616282
:10B5FC006C696E672074686520424C4520737461D9
:10B60C00636B2E004E6F206164766572746973698A
:10B61C006E67206E616D6520666F756E6400536594
:10B62C007474696E6720616476206E616D653A2072
:10B63C0025732C206C656E6774683A202564005560
:10B64C0073696E672064656661756C7420616476DD
:10B65C006572746973696E67206E616D6500424C2A
:10B66C004520444655207472616E73706F7274205D
:10B67C00696E697469616C697A65642E006E7266B4
:10B68C005F6466755F626C650050EADA308883B877
:10B69C009F604F15F30000C98E00000000000000F1
:10B6AC00000000000338FDD870470C000C000000AF
:10B6BC005802777269746500657261736500466C37
:10B6CC0061736820257320737563636573733A2007
:10B6DC00616464723D25702C2070656E64696E67C0
:10B6EC0020256400466C61736820257320666169AF
:10B6FC006C6564202830782578293A20616464725E
:10B70C003D25702C206C656E3D3078257820627953
:10B71C007465732C2070656E64696E6720256400F7
:10B72C00496E697469616C697A696E67206E7266BC
:10B73C005F6673746F726167655F736420626163C7
:10B74C006B656E642E00496E697469616C697A6907
:10B75C006E67206E72665F6673746F726167655F89
:10B76C006E766D63206261636B656E642E006E7223
:10B77C00665F6673746F726167655F777269746513
:10B78C0028616464723D25702C207372633D2570B2
:10B79C002C206C656E3D2564206279746573292CB0
:10B7AC002071756575652075736167653A20256430
:10B7BC00006E72665F6673746F726167655F777235
:10B7CC006974652829206661696C656420776974E1
:10B7DC0068206572726F7220307825782E006E7238
:10B7EC00665F6673746F726167655F6572617365BE
:10B7FC0028616464723D307825702C206C656E3D38
:10B80C002564207061676573292C207175657565D9
:10B81C002075736167653A202564006E72665F66F9
:10B82C0073746F726167655F657261736528292037
:10B83C006661696C65642077697468206572726FE3
:10B84C007220307825782E006E72665F6466755FA4
:10B85C00666C61736800416C6C20666C6173682067
:10B86C006F7065726174696F6E73206861766520A4
:10B87C00636F6D706C657465642E2044465520634F
:10B88C006F6D706C657465642E004661696C6564DF
:10B89C0020746F207363686564756C65206F626AD1
:10B8AC0065637420657865637574653A2030782516
:10B8BC00782E0057686F6C65206669726D776172BF
:10B8CC006520696D6167652072656365697665647D
:10B8DC002E20506F737476616C69646174696E6745
:10B8EC002E00526571756573742068616E646C69A5
:10B8FC006E6720636F6D706C6574652E2052657376
:10B90C00756C743A203078257800443A5C576F7225
:10B91C006B5F4A616B756A615C5355484F5F494D6B
:10B92C004147455C31315F454D455247454E435982
:10B93C005F5357495443485C23544F4F4C535C73EB
:10B94C0072635F32303231313231395C30315F64A5
:10B95C0066755F626C652E32303231313231395C52
:10B96C00636F6D706F6E656E74735C6C696272611F
:10B97C00726965735C626F6F746C6F616465725C25
:10B98C006466755C6E72665F6466755F7265715F26
:10B99C0068616E646C65722E630048616E646C65E0
:10B9AC00204E52465F4446555F4F505F52454345CB
:10B9BC004950545F4E4F5449465F534554004861BB
:10B9CC006E646C65204E52465F4446555F4F505F27
:10B9DC0041424F52540048616E646C65204E524691
:10B9EC005F4446555F4F505F4F424A4543545F4357
:10B9FC0052454154452028636F6D6D616E6429007A
:10BA0C0048616E646C65204E52465F4446555F4FEC
:10BA1C00505F4352435F4745542028636F6D6D61FF
:10BA2C006E64290048616E646C65204E52465F441A
:10BA3C0046555F4F505F4F424A4543545F575249FA
:10BA4C0054452028636F6D6D616E64290048616EEA
:10BA5C00646C65204E52465F4446555F4F505F4FB5
:10BA6C00424A4543545F4558454355544520286345
:10BA7C006F6D6D616E64290057726974696E672011
:10BA8C0076616C696420696E697420636F6D6D6199
:10BA9C006E6420746F20666C6173682E0048616E52
:10BAAC00646C65204E52465F4446555F4F505F4F65
:10BABC00424A4543545F53454C4543542028636FD9
:10BACC006D6D616E64290048616E646C65204E5228
:10BADC00465F4446555F4F505F4F424A4543545F63
:10BAEC0043524541544520286461746129004361E7
:10BAFC006E6E6F742063726561746520646174612D
:10BB0C00206F626A65637420776974686F7574203E
:10BB1C0076616C696420696E697420636F6D6D6108
:10BB2C006E64004F626A6563742073697A65206382
:10BB3C00616E6E6F7420626520302E004F626A65F4
:10BB4C0063742073697A65206D7573742062652047
:10BB5C007061676520616C69676E656400496E761B
:10BB6C00616C69642073697A6520666F72206F62FC
:10BB7C006A6563742028746F6F206C617267652925
:10BB8C00004372656174696E6720746865206F622A
:10BB9C006A65637420776974682073697A652030EC
:10BBAC00782530387820776F756C64206F766572E5
:10BBBC00666C6F77206669726D7761726520736948
:10BBCC007A652E204F666673657420697320307811
:10BBDC002530387820616E64206669726D776172E9
:10BBEC00652073697A652069732030782530387840
:10BBFC002E004572617365206F7065726174696F98
:10BC0C006E206661696C6564004372656174696E6F
:10BC1C0067206F626A656374207769746820736942
:10BC2C007A653A2025642E204F66667365743A2037
:10BC3C003078253038782C204352433A2030782500
:10BC4C003038780048616E646C65204E52465F4413
:10BC5C0046555F4F505F4F424A4543545F575249D8
:10BC6C0054452028646174612900577269746520F9
:10BC7C007265717565737420746F6F206C6F6E676D
:10BC8C000048616E646C65204E52465F4446555FB9
:10BC9C004F505F4352435F474554202864617461A1
:10BCAC0029004F66667365743A25642C2043524311
:10BCBC003A3078253038780048616E646C65204ED7
:10BCCC0052465F4446555F4F505F4F424A4543547E
:10BCDC005F455845435554452028646174612900DB
:10BCEC00496E76616C696420646174612E2065789C
:10BCFC007065637465643A2025642C20676F743A10
:10BD0C002025640048616E646C65204E52465F4489
:10BD1C0046555F4F505F4F424A4543545F53454C25
:10BD2C004543542028646174612900637263203D8B
:10BD3C0020307825782C206F6666736574203D2042
:10BD4C00307825782C206D61785F73697A65203D99
:10BD5C00203078257800496E76616C6964206F62BA
:10BD6C006A656374207479706520696E20726571E0
:10BD7C00756573742E00496E76616C6964206F7002
:10BD8C00636F64652072656365697665643A20301B
:10BD9C007825782E005363686564756C6572207223
:10BDAC00616E206F7574206F6620737061636521FE
:10BDBC00006E72665F6466755F7265715F68616E56
:10BDCC00646C65720044657374696E6174696F6E3E
:10BDDC002073657474696E67732061726520696481
:10BDEC00656E746963616C20746F20736F75726318
:10BDFC00652C207772697465206E6F74206E656592
:10BE0C006465642E20536B697070696E672E0057E1
:10BE1C00726974696E672073657474696E67732ECA
:10BE2C002E2E0045726173696E67206F6C642073EF
:10BE3C00657474696E67732061743A2030782530AC
:10BE4C00387800436F756C64206E6F742065726176
:10BE5C007365207468652073657474696E677320EC
:10BE6C00706167652100436F756C64206E6F742080
:10BE7C007772697465207468652044465520736533
:10BE8C007474696E677320706167652100557369FE
:10BE9C006E672073657474696E6773207061676573
:10BEAC002E00436F7079696E6720666F72626964E9
:10BEBC0064656E2070617274732066726F6D20629F
:10BECC0061636B757020706167652E0052657374C9
:10BEDC006F72696E672073657474696E6773206620
:10BEEC00726F6D206261636B75702073696E636530
:10BEFC00207468652073657474696E677320706153
:10BF0C00676520636F6E74656E7473206172652053
:10BF1C00696E76616C6964202843524320657272A5
:10BF2C006F72292E00526573657474696E67206296
:10BF3C006F6F746C6F616465722073657474696E75
:10BF4C0067732073696E6365206E656974686572CA
:10BF5C00207468652073657474696E6773207061F2
:10BF6C006765206E6F7220746865206261636B7503
:10BF7C0070206172652076616C696420284352439D
:10BF8C00206572726F72292E004F6C642073657479
:10BF9C0074696E677320706167652064657465638E
:10BFAC007465642E20557067726164696E672069D0
:10BFBC006E666F2E004261636B696E672075702030
:10BFCC0073657474696E6773207061676520746F34
:10BFDC00206164647265737320307825782E004478
:10BFEC003A5C576F726B5F4A616B756A615C535553
:10BFFC00484F5F494D4147455C31315F454D455296
:10C00C0047454E43595F5357495443485C23544F5B
:10C01C004F4C535C7372635F323032313132313991
:10C02C005C30315F6466755F626C652E3230323124
:10C03C00313231395C636F6D706F6E656E74735C29
:10C04C006C69627261726965735C626F6F746C6F3C
:10C05C00616465725C6466755C6E72665F6466755D
:10C06C005F73657474696E67732E6300436F756CD0
:10C07C0064206E6F7420706572666F726D206261E1
:10C08C00636B7570206F6620626F6F746C6F616488
:10C09C0065722073657474696E67732120457272C2
:10C0AC006F723A20307825780043616C6C696E674A
:10C0BC00206E72665F6466755F73657474696E6713
:10C0CC00735F696E697428292E2E2E006E72665F5E
:10C0DC006466755F666C6173685F696E6974282944
:10C0EC00206661696C65642077697468206572727A
:10C0FC006F723A202578006E72665F6466755F73A6
:10C10C00657474696E67735F77726974655F616E6D
:10C11C00645F6261636B75702829206661696C6568
:10C12C00642077697468206572726F723A20257882
:10C13C00006E72665F6466755F73657474696E67B2
:10C14C00730045726173696E672073657474696EF0
:10C15C0067732070616765206164646974696F6ED0
:10C16C00616C20646174612E006E72665F6466752A
:10C17C005F73657474696E67735F73766369004986
:10C18C006E697469616C697A696E67207472616E2C
:10C19C0073706F7274732028666F756E643A202505
:10C1AC006429004661696C656420746F20696E694E
:10C1BC007469616C697A65207472616E73706F72E8
:10C1CC00742025642C206572726F722025640053D4
:10C1DC0068757474696E6720646F776E2074726111
:10C1EC006E73706F7274732028666F756E643A206C
:10C1FC00256429004661696C656420746F2073683E
:10C20C007574646F776E207472616E73706F727474
:10C21C002025642C206572726F7220256400456E97
:10C22C00746572206E72665F6466755F63616368C5
:10C23C00655F707265706172652829007265717531
:10C24C00697265645F73697A653A20307825782E57
:10C25C0000747275650066616C73650073696E6756
:10C26C006C655F62616E6B3A2025732E006B6565A1
:10C27C00705F6170703A2025732E006B6565705F7E
:10C28C00736F66746465766963653A2025732E0056
:10C29C0053445F50524553454E543A2025732E005B
:10C2AC0042616E6B20636F6E74656E74733A0042FC
:10C2BC00616E6B203020636F64653A2030782530D6
:10C2CC0032783A2053697A653A20307825780042E2
:10C2DC00616E6B203120636F64653A2030782530B5
:10C2EC0032783A2053697A653A20307825780044C0
:10C2FC003A5C576F726B5F4A616B756A615C535540
:10C30C00484F5F494D4147455C31315F454D455282
:10C31C0047454E43595F5357495443485C23544F48
:10C32C004F4C535C7372635F32303231313231397E
:10C33C005C30315F6466755F626C652E3230323111
:10C34C00313231395C636F6D706F6E656E74735C16
:10C35C006C69627261726965735C626F6F746C6F29
:10C36C00616465725C6466755C6E72665F6466754A
:10C37C005F7574696C732E6300706173733A20255A
:10C38C00642E0063616368655F61646472657373D6
:10C39C003A20307825782E0063616368655F746F8E
:10C3AC006F5F736D616C6C3A2025732E006B656545
:10C3BC00705F6669726D776172653A2025732E0025
:10C3CC0064656C6574655F6D6F72653A2025732EBC
:10C3DC000041626F7274696E672E2043616E6E6FDE
:10C3EC007420666974206E6577206669726D77615A
:10C3FC007265206F6E2064657669636500496E76A0
:10C40C00616C69646174696E67206170702E00489C
:10C41C00616E646C65723A20496E76616C69642059
:10C42C0070726F746F636F6C2062756666657220D4
:10C43C006D5F70625F73747265616D0048616E64EC
:10C44C006C65723A20496E76616C696420696E691C
:10C45C007420636F6D6D616E642E0048616E646C48
:10C46C0065723A20496E76616C69642070726F74E3
:10C47C006F636F6C20627566666572206D5F7062AB
:10C48C005F73747265616D2028696E697420636FC7
:10C49C006D6D616E642900424C2073697A652028A9
:10C4AC00256429206F766572206C696D697420286B
:10C4BC0025642900496E6974207061636B65742072
:10C4CC00646F6573206E6F7420636F6E7461696E38
:10C4DC002076616C6964206669726D776172652083
:10C4EC0073697A650050423A20496E697420706114
:10C4FC00636B65742064617461206C656E3A2025F1
:10C50C006400443A5C576F726B5F4A616B756A6189
:10C51C005C5355484F5F494D4147455C31315F4550
:10C52C004D455247454E43595F5357495443485C18
:10C53C0023544F4F4C535C7372635F323032313142
:10C54C003231395C30315F6466755F626C652E32F6
:10C55C00303231313231395C636F6D706F6E656EB4
:10C56C0074735C6C69627261726965735C626F6F23
:10C57C00746C6F616465725C6466755C6E72665F28
:10C58C006466755F76616C69646174696F6E2E6345
:10C59C00005369676E617475726520726571756997
:10C5AC007265642E20436865636B696E67207369DE
:10C5BC00676E61747572652E004E6F207369676EBD
:10C5CC00617475726520666F756E642E00496E76A7
:10C5DC00616C6964207369676E617475726520742F
:10C5EC007970650043616C63756C6174696E67206A
:10C5FC006861736820286C656E3A202564290056A2
:10C60C006572696679207369676E6174757265000D
:10C61C005369676E6174757265206661696C6564D7
:10C62C0020286572725F636F64653A2030782578D4
:10C63C0029005369676E61747572653A00486173BD
:10C64C00683A005075626C6963204B65793A004911
:10C65C006D616765207665726966696564006D61F8
:10C66C006A6F72006D696E6F7200536F6674446509
:10C67C0076696365207570646174652069732061E7
:10C68C002025732076657273696F6E2075706461F6
:10C69C0074652E2043757272656E743A2025642E73
:10C6AC00204E65773A2025642E0048617368207609
:10C6BC006572696669636174696F6E2E207374614B
:10C6CC00727420616464726573733A2030782578D3
:10C6DC002C2073697A653A203078257800436F7581
:10C6EC006C64206E6F742072756E206861736820A4
:10C6FC00766572696669636174696F6E202865720C
:10C70C00725F636F64652030782578292E0048614C
:10C71C00736820766572696669636174696F6E20EF
:10C72C006661696C65642E00457870656374656438
:10C73C0020465720686173683A0041637475616CD8
:10C74C0020465720686173683A00496E697420630B
:10C75C006F6D6D616E64206C6172676572207468B8
:10C76C00616E2065787065637465642E0050726527
:10C77C0076616C69646174696F6E206661696C6561
:10C78C00642E00496E697420636F6D6D616E643A3E
:10C79C0000457865637574652077697468206661F7
:10C7AC00756C7479206F66667365740043616E27CF
:10C7BC00742066696E6420726F6F6D20666F7220D4
:10C7CC007570646174650057726974652061646486
:10C7DC00726573732073657420746F203078253004
:10C7EC003878004661696C656420746F20646563F9
:10C7FC006F646520696E6974207061636B65740089
:10C80C0043524320636865636B206F6620617070D0
:10C81C00206661696C65642E2052657475726E2099
:10C82C002564006E72665F63727970746F5F686105
:10C83C0073685F63616C63756C617465282920662D
:10C84C0061696C65642077697468206572726F72B7
:10C85C0020257300496E76616C696420626F6F7479
:10C86C002076616C69646174696F6E20747970658F
:10C87C003A20256400496E76616C69646174696E56
:10C88C0067206F6C64206170706C69636174696F90
:10C89C006E20696E2062616E6B20302E00546865CC
:10C8AC0020536F667444657669636520646F6573A5
:10C8BC00206E6F7420636F6E7461696E207468658E
:10C8CC00206D61676963206E756D626572206964A5
:10C8DC00656E74696679696E67206974206173206E
:10C8EC006120536F66744465766963652E005468E5
:10C8FC006520536F66744465766963652073697A45
:10C90C006520696E2074686520696E666F2073748B
:10C91C007275637420697320746F6F20736D616C12
:10C92C006C20636F6D706172656420776974682028
:10C93C007468652073697A65207265706F727465AE
:10C94C006420696E2074686520696E697420636F59
:10C95C006D6D616E642E00546865206E6577205392
:10C96C006F6674446576696365206973206F662011
:10C97C006120646966666572656E742066616D69B6
:10C98C006C79207468616E207468652070726573B0
:10C99C00656E7420536F66744465766963652E20EA
:10C9AC00436F6D7061746962696C6974792063613D
:10C9BC006E6E6F742062652067756172616E74654E
:10C9CC0065642E00496E76616C69646174696E678A
:10C9DC0020617070206265636175736520697420D5
:10C9EC00697320696E636F6D70617469626C652028
:10C9FC00776974682074686520536F667444657633
:10CA0C006963652E004D616A6F7220534420757006
:10CA1C006461746520627574206E6F20424C2E2008
:10CA2C0041626F727420746F2061766F6964206943
:10CA3C006E636170616369746174696E6720746898
:10CA4C006520424C2E00426F6F742076616C6964D5
:10CA5C006174696F6E206F6620626F6F746C6F61AA
:10CA6C00646572206973206E6F7420737570706FBB
:10CA7C007274656420616E642077696C6C206265E9
:10CA8C002069676E6F7265642E006E72665F6466F5
:10CA9C00755F76616C69646174696F6E00443A5CB1
:10CAAC00576F726B5F4A616B756A615C5355484F87
:10CABC005F494D4147455C31315F454D45524745D6
:10CACC004E43595F5357495443485C23544F4F4C82
:10CADC00535C7372635F32303231313231395C30D6
:10CAEC00315F6466755F626C652E32303231313283
:10CAFC0031395C636F6D706F6E656E74735C6C69ED
:10CB0C00627261726965735C626F6F746C6F616481
:10CB1C0065725C6466755C6E72665F6466755F7682
:10CB2C0065725F76616C69646174696F6E2E630007
:10CB3C00496E76616C6964206669726D77617265A5
:10CB4C0020747970652E00496E76616C696420687A
:10CB5C0061736820747970652E004E6F20485720E1
:10CB6C0076657273696F6E2E004661756C747920F0
:10CB7C0048572076657273696F6E2E00534420728D
:10CB8C006571206E6F74206D65742E00465720768B
:10CB9C00657273696F6E20746F6F206C6F772E00E7
:10CBAC0046572076657273696F6E206D6973736971
:10CBBC006E672E006E72665F6466755F7665725F77
:10CBCC0076616C69646174696F6E006E72665F7316
:10CBDC006468000100000700709607007896070053
:10CBEC0008000000809607009096070008000000DF
:10CBFC0078960700809607000800000073645F6257
:10CC0C006C655F6366675F73657428292072657451
:10CC1C0075726E6564202573207768656E2061746B
:10CC2C0074656D7074696E6720746F207365742001
:10CC3C00424C455F434F4E4E5F4346475F47415022
:10CC4C002E0073645F626C655F6366675F73657407
:10CC5C0028292072657475726E656420257320779F
:10CC6C0068656E20617474656D7074696E6720748C
:10CC7C006F2073657420424C455F4741505F4346BB
:10CC8C00475F524F4C455F434F554E542E007364D3
:10CC9C005F626C655F6366675F73657428292072D9
:10CCAC00657475726E6564202573207768656E20D7
:10CCBC00617474656D7074696E6720746F20736530
:10CCCC007420424C455F434F4E4E5F4346475F478F
:10CCDC004154542E0073645F626C655F6366675FDA
:10CCEC0073657428292072657475726E65642025CD
:10CCFC0073207768656E20617474656D7074696EED
:10CD0C006720746F2073657420424C455F434F4D10
:10CD1C004D4F4E5F4346475F56535F555549442E22
:10CD2C000073645F626C655F6366675F736574282C
:10CD3C00292072657475726E65642025732077687E
:10CD4C00656E20617474656D7074696E6720746FA4
:10CD5C002073657420424C455F47415454535F43E4
:10CD6C0046475F415454525F5441425F53495A45C0
:10CD7C002E0073645F626C655F6366675F736574D6
:10CD8C0028292072657475726E656420257320776E
:10CD9C0068656E20617474656D7074696E6720745B
:10CDAC006F2073657420424C455F47415454535F68
:10CDBC004346475F534552564943455F4348414EAE
:10CDCC004745442E00496E73756666696369656EE6
:10CDDC00742052414D20616C6C6F636174656420EA
:10CDEC00666F722074686520536F6674446576694B
:10CDFC0063652E004368616E676520746865205218
:10CE0C00414D207374617274206C6F636174696F2F
:10CE1C006E2066726F6D203078257820746F20300C
:10CE2C007825782E004D6178696D756D2052414DD5
:10CE3C002073697A6520666F72206170706C69630B
:10CE4C006174696F6E20697320307825782E0073B9
:10CE5C00645F626C655F656E61626C652829207227
:10CE6C00657475726E65642025732E006E72665F34
:10CE7C007364685F626C65006896070070960700C3
:10CE8C00080000006E72665F7364685F736F630006
:10CE9C0090960700989607000800000043000000D9
:10CEAC00504F5349580000002020202020202020E3
:10CEBC0020682828282820202020202020202020FE
:10CECC00202020202020202048101010101010109E
:10CEDC0010101010101010108484848484848484A6
:10CEEC0084841010101010101081818181818101B7
:10CEFC000101010101010101010101010101010116
:10CF0C0001010110101010101082828282828202A4
:10CF1C0002020202020202020202020202020202E5
:10CF2C000202021010101020000703200417020147
:10CF3C000857104080000000A8CE0700ACCF0700B7
:10CF4C00C0D0070053756E004D6F6E0054756500B0
:10CF5C00576564005468750046726900536174002B
:10CF6C00000000004A616E00466562004D6172006F
:10CF7C00417072004D6179004A756E004A756C0003
:10CF8C0041756700536570004F6374004E6F7600F7
:10CF9C004465630000000000414D00504D0000004E
:10CFAC00E4D00700E0D00700E0D00700E0D0070095
:10CFBC00E0D00700E0D00700E0D00700E0D0070089
:10CFCC00E0D00700E0D00700FFFFFFFFFFFFFFFFEF
:10CFDC00FFFFFFFFFFFF000020D0070050CF07002E
:10CFEC005CD0070070CF0700A4CF070004D0070067
:10CFFC00B4D0070010D00700256D2F25642F25799C
:10D00C000000000025612025622025652025542084
:10D01C002559000053756E646179004D6F6E646123
:10D02C00790054756573646179005765646E657336
:10D03C006461790054687572736461790046726931
:10D04C006461790053617475726461790000000049
:10D05C004A616E75617279004665627275617279AA
:10D06C00004D6172636800417072696C004D6179AA
:10D07C00004A756E65004A756C7900417567757369
:10D08C00740053657074656D626572004F63746FE4
:10D09C00626572004E6F76656D6265720044656301
:10D0AC00656D62657200000025483A254D3A25539E
:10D0BC0000000000299307004593070051930700D7
:10D0CC005D93070079930700859307009193070000
:0AD0DC009F930700000000002E00E3
:10D0E80000000000FF000000000000000000000039
:10D0F8000000000000000000000000000000000028
:10D10800000000000100000084590020945900200C
:10D118000090D003FF00FFFF0100000000E00700BF
:10D1280044CF070044CF070044CF070044CF07008F
:04D1380044CF0700D9
:020000020000FC
:020000041000EA
:0410140000100700C1
:0410180000E00700ED
:040000037000135D19
:00000001FF
